******************************************************************************
               TMS320C6x Linker PC v7.3.1                      
******************************************************************************
>> Linked Fri May 18 10:11:02 2012

OUTPUT FILE NAME:   <TestAppEncoder.out>
ENTRY POINT SYMBOL: "_c_int00"  address: 0c020480


MEMORY CONFIGURATION

         name            origin    length      used     unused   attr    fill
----------------------  --------  ---------  --------  --------  ----  --------
  L2SRAM                00800000   00060000  0000e7ad  00051853  RW X
  MSMCSRAM              0c000000   00400000  00024040  003dbfc0  RW X
  ERAM                  80000000   08000000  022da6e8  05d25918  RWIX


SEGMENT ALLOCATION MAP

run origin  load origin   length   init length attrs members
----------  ----------- ---------- ----------- ----- -------
00800000    00800000    000047c8   000047c8    rw-
  00800000    00800000    000047c8   000047c8    rw- .const.1
008047d0    008047d0    000000e8   000000e8    r--
  008047d0    008047d0    000000e8   000000e8    r-- .const.2
008048c0    008048c0    00000048   00000048    r--
  008048c0    008048c0    00000048   00000048    r-- .const.3
00804910    00804910    000006a8   000006a8    r--
  00804910    00804910    000006a8   000006a8    r-- .const.4
00804fc0    00804fc0    00000088   00000088    r--
  00804fc0    00804fc0    00000088   00000088    r-- .const.5
00805050    00805050    00000007   00000007    r--
  00805050    00805050    00000007   00000007    r-- .const.6
00805060    00805060    00000006   00000006    r--
  00805060    00805060    00000006   00000006    r-- .const.7
00805070    00805070    00000004   00000004    r--
  00805070    00805070    00000004   00000004    r-- .const.8
00805080    00805080    00000004   00000004    r--
  00805080    00805080    00000004   00000004    r-- .const.9
00805088    00805088    00002000   00000000    rw-
  00805088    00805088    00002000   00000000    rw- .stack
00807090    00807090    000016f8   000016f8    rw-
  00807090    00807090    000016f8   000016f8    rw- .fardata.1
00808790    00808790    00000018   00000018    rw-
  00808790    00808790    00000018   00000018    rw- .fardata.2
008087b0    008087b0    00000014   00000014    rw-
  008087b0    008087b0    00000014   00000014    rw- .fardata.3
008087d0    008087d0    00000014   00000014    rw-
  008087d0    008087d0    00000014   00000014    rw- .fardata.4
008087f0    008087f0    00000028   00000028    rw-
  008087f0    008087f0    00000028   00000028    rw- .fardata.5
00808820    00808820    00000008   00000008    rw-
  00808820    00808820    00000008   00000008    rw- .fardata.6
00808830    00808830    00000008   00000008    rw-
  00808830    00808830    00000008   00000008    rw- .fardata.7
00808840    00808840    00000004   00000004    rw-
  00808840    00808840    00000004   00000004    rw- .fardata.8
00808850    00808850    00000004   00000004    rw-
  00808850    00808850    00000004   00000004    rw- .fardata.9
00808860    00808860    00000004   00000004    rw-
  00808860    00808860    00000004   00000004    rw- .fardata.10
00808870    00808870    00000004   00000004    rw-
  00808870    00808870    00000004   00000004    rw- .fardata.11
00808880    00808880    00000004   00000004    rw-
  00808880    00808880    00000004   00000004    rw- .fardata.12
00808888    00808888    00000800   00000000    rw-
  00808888    00808888    00000800   00000000    rw- .taskStackSection
00809088    00809088    00000200   00000200    rw-
  00809088    00809088    00000200   00000200    rw- .args
00809288    00809288    000001a4   000001a4    r--
  00809288    00809288    000001a4   000001a4    r-- .switch
0080942c    0080942c    00000120   00000000    rw-
  0080942c    0080942c    00000120   00000000    rw- .cio
00809550    00809550    00000030   00000000    rw-
  00809550    00809550    00000030   00000000    rw- .bss
00809580    00809580    00000010   00000010    rw-
  00809580    00809580    00000010   00000010    rw- .neardata
00809590    00809590    000052e8   000052e8    r--
  00809590    00809590    000052e8   000052e8    r-- .cinit
0c000000    0c000000    00023e40   00023e40    r-x
  0c000000    0c000000    00023e40   00023e40    r-x .text
0c024000    0c024000    00000200   00000200    r-x
  0c024000    0c024000    00000200   00000200    r-x .vecs
80000000    80000000    01f166e8   00000000    rw-
  80000000    80000000    01f166e8   00000000    rw- .far
81f166f0    81f166f0    003a4000   00000000    rw-
  81f166f0    81f166f0    00384000   00000000    rw- .ccdData
  8229a6f0    8229a6f0    00020000   00000000    rw- .bitsData
822ba700    822ba700    00020000   00000000    rw-
  822ba700    822ba700    00020000   00000000    rw- .ref_buffer


SECTION ALLOCATION MAP

 output                                  attributes/
section   page    origin      length       input sections
--------  ----  ----------  ----------   ----------------
.init_array 
*          0    00800000    00000000     UNINITIALIZED

.cinit     0    80000000    00000000     UNINITIALIZED

.init_array 
*          0    00800000    00000000     UNINITIALIZED

xdc.meta   0    00800000    00000178     COPY SECTION
                  00800000    00000178     JpegEncApp6678.pe66.obj (xdc.meta)

.const.1   0    00800000    000047c8     
                  00800000    00002286     JpegEncApp6678.pe66.obj (.const:xdc_runtime_Text_charTab__A)
                  00802286    00000002     --HOLE--
                  00802288    00000004     JpegEncApp6678.pe66.obj (.const:ti_sdo_ipc_gates_GateHWSem_reservedMaskArr__C)
                  0080228c    00000004     JpegEncApp6678.pe66.obj (.const:ti_sdo_ipc_interfaces_IGateMPSupport_Interface__BASE__C)
                  00802290    1fff8ad4     jpgealg_ti.le66 (.const:JPEGIENC_TI_dSect)
                  008032f2    00000002     --HOLE--
                  008032f4    00000774     TestAppEncoder.obj (.const)
                  00803a68    000004f6     JpegEncApp6678.pe66.obj (.const)
                  00803f5e    00000002     --HOLE--
                  00803f60    00000400     JpegEncApp6678.pe66.obj (.const:ti_sysbios_family_c66_Cache_marvalues__C)
                  00804360    000001a8     alg_malloc.obj (.const)
                  00804508    00000004     JpegEncApp6678.pe66.obj (.const:xdc_runtime_IGateProvider_Interface__BASE__C)
                  0080450c    00000004     JpegEncApp6678.pe66.obj (.const:xdc_runtime_IHeap_Interface__BASE__C)
                  00804510    0000014c     JpegEncApp6678.pe66.obj (.const:xdc_runtime_Text_nodeTab__A)
                  0080465c    00000004     JpegEncApp6678.pe66.obj (.const:xdc_runtime_IModule_Interface__BASE__C)
                  00804660    00000101     rts6600_elf.lib : ctype.obj (.const:_ctypes_)
                  00804761    00000003     --HOLE--
                  00804764    00000064     TestAppConfigParser.obj (.const)

.const.2   0    008047d0    000000e8     
                  008047d0    00000050     rts6600_elf.lib : strtod.obj (.const:digits)
                  00804820    00000050                     : strtold.obj (.const:digits)
                  00804870    00000048                     : strtod.obj (.const:powerof10)

.const.3   0    008048c0    00000048     
                  008048c0    00000048     rts6600_elf.lib : strtold.obj (.const:powerof10)

.const.4   0    00804910    000006a8     
                  00804910    0000003c     JpegEncApp6678.pe66.obj (.const:xdc_runtime_Startup_sfxnTab__A)
                  0080494c    00000038     JpegEncApp6678.pe66.obj (.const:ti_sysbios_knl_Task_Object__PARAMS__C)
                  00804984    00000034     JpegEncApp6678.pe66.obj (.const:ti_sdo_ipc_GateMP_Object__PARAMS__C)
                  008049b8    00000030     JpegEncApp6678.pe66.obj (.const:ti_sdo_ipc_heaps_HeapMemMP_Object__PARAMS__C)
                  008049e8    0000002c     JpegEncApp6678.pe66.obj (.const:ti_sdo_ipc_gates_GateHWSem_Module__FXNS__C)
                  00804a14    0000002c     JpegEncApp6678.pe66.obj (.const:ti_sdo_ipc_gates_GateMPSupportNull_Module__FXNS__C)
                  00804a40    0000002c     JpegEncApp6678.pe66.obj (.const:ti_sdo_ipc_gates_GatePeterson_Module__FXNS__C)
                  00804a6c    00000028     JpegEncApp6678.pe66.obj (.const:ti_sdo_ipc_heaps_HeapMemMP_Module__FXNS__C)
                  00804a94    00000028     JpegEncApp6678.pe66.obj (.const:ti_sysbios_heaps_HeapMem_Module__FXNS__C)
                  00804abc    00000024     JpegEncApp6678.pe66.obj (.const:ti_sdo_ipc_gates_GateHWSem_Object__PARAMS__C)
                  00804ae0    00000024     JpegEncApp6678.pe66.obj (.const:ti_sdo_ipc_gates_GateMPSupportNull_Object__PARAMS__C)
                  00804b04    00000024     JpegEncApp6678.pe66.obj (.const:ti_sdo_ipc_gates_GatePeterson_Object__PARAMS__C)
                  00804b28    00000024     JpegEncApp6678.pe66.obj (.const:ti_sysbios_gates_GateAll_Module__FXNS__C)
                  00804b4c    00000024     JpegEncApp6678.pe66.obj (.const:ti_sysbios_gates_GateMutexPri_Module__FXNS__C)
                  00804b70    00000024     JpegEncApp6678.pe66.obj (.const:ti_sysbios_gates_GateMutex_Module__FXNS__C)
                  00804b94    00000024     JpegEncApp6678.pe66.obj (.const:ti_sysbios_gates_GateSwi_Module__FXNS__C)
                  00804bb8    00000024     JpegEncApp6678.pe66.obj (.const:ti_sysbios_knl_Clock_Object__PARAMS__C)
                  00804bdc    00000024     JpegEncApp6678.pe66.obj (.const:ti_sysbios_knl_Semaphore_Object__PARAMS__C)
                  00804c00    00000024     JpegEncApp6678.pe66.obj (.const:xdc_runtime_GateNull_Module__FXNS__C)
                  00804c24    00000024     JpegEncApp6678.pe66.obj (.const:xdc_runtime_knl_GateThread_Module__FXNS__C)
                  00804c48    00000023     rts6600_elf.lib : _printfi.obj (.const)
                  00804c6b    00000001     --HOLE--
                  00804c6c    00000020     JpegEncApp6678.pe66.obj (.const:ti_sdo_ipc_GateMP_Object__DESC__C)
                  00804c8c    00000020     JpegEncApp6678.pe66.obj (.const:ti_sdo_ipc_Notify_Object__DESC__C)
                  00804cac    00000020     JpegEncApp6678.pe66.obj (.const:ti_sdo_ipc_gates_GateHWSem_Object__DESC__C)
                  00804ccc    00000020     JpegEncApp6678.pe66.obj (.const:ti_sdo_ipc_gates_GateMPSupportNull_Object__DESC__C)
                  00804cec    00000020     JpegEncApp6678.pe66.obj (.const:ti_sdo_ipc_gates_GatePeterson_Object__DESC__C)
                  00804d0c    00000020     JpegEncApp6678.pe66.obj (.const:ti_sdo_ipc_heaps_HeapMemMP_Object__DESC__C)
                  00804d2c    00000020     JpegEncApp6678.pe66.obj (.const:ti_sdo_utils_List_Object__DESC__C)
                  00804d4c    00000020     JpegEncApp6678.pe66.obj (.const:ti_sysbios_gates_GateAll_Object__DESC__C)
                  00804d6c    00000020     JpegEncApp6678.pe66.obj (.const:ti_sysbios_gates_GateMutexPri_Object__DESC__C)
                  00804d8c    00000020     JpegEncApp6678.pe66.obj (.const:ti_sysbios_gates_GateMutex_Object__DESC__C)
                  00804dac    00000020     JpegEncApp6678.pe66.obj (.const:ti_sysbios_gates_GateSwi_Object__DESC__C)
                  00804dcc    00000020     JpegEncApp6678.pe66.obj (.const:ti_sysbios_heaps_HeapMem_Object__DESC__C)
                  00804dec    00000020     JpegEncApp6678.pe66.obj (.const:ti_sysbios_heaps_HeapMem_Object__PARAMS__C)
                  00804e0c    00000020     JpegEncApp6678.pe66.obj (.const:ti_sysbios_knl_Clock_Object__DESC__C)
                  00804e2c    00000020     JpegEncApp6678.pe66.obj (.const:ti_sysbios_knl_Queue_Object__DESC__C)
                  00804e4c    00000020     JpegEncApp6678.pe66.obj (.const:ti_sysbios_knl_Semaphore_Object__DESC__C)
                  00804e6c    00000020     JpegEncApp6678.pe66.obj (.const:ti_sysbios_knl_Task_Object__DESC__C)
                  00804e8c    00000020     JpegEncApp6678.pe66.obj (.const:ti_sysbios_xdcruntime_GateThreadSupport_Object__DESC__C)
                  00804eac    00000020     JpegEncApp6678.pe66.obj (.const:xdc_runtime_GateNull_Object__DESC__C)
                  00804ecc    00000020     JpegEncApp6678.pe66.obj (.const:xdc_runtime_knl_GateThread_Object__DESC__C)
                  00804eec    00000004     --HOLE--
                  00804ef0    0000001e     JpegEncApp6678.pe66.obj (.const:xdc_runtime_Startup_sfxnRts__A)
                  00804f0e    00000002     --HOLE--
                  00804f10    00000018     JpegEncApp6678.pe66.obj (.const:ti_sdo_ipc_Notify_Object__PARAMS__C)
                  00804f28    00000018     JpegEncApp6678.pe66.obj (.const:ti_sdo_utils_List_Object__PARAMS__C)
                  00804f40    00000018     JpegEncApp6678.pe66.obj (.const:ti_sysbios_gates_GateAll_Object__PARAMS__C)
                  00804f58    00000018     JpegEncApp6678.pe66.obj (.const:ti_sysbios_gates_GateMutexPri_Object__PARAMS__C)
                  00804f70    00000018     JpegEncApp6678.pe66.obj (.const:ti_sysbios_gates_GateMutex_Object__PARAMS__C)
                  00804f88    00000018     JpegEncApp6678.pe66.obj (.const:ti_sysbios_gates_GateSwi_Object__PARAMS__C)
                  00804fa0    00000018     JpegEncApp6678.pe66.obj (.const:ti_sysbios_knl_Queue_Object__PARAMS__C)

.const.5   0    00804fc0    00000088     
                  00804fc0    00000018     JpegEncApp6678.pe66.obj (.const:ti_sysbios_knl_Task_hooks__A)
                  00804fd8    00000018     JpegEncApp6678.pe66.obj (.const:ti_sysbios_xdcruntime_GateThreadSupport_Object__PARAMS__C)
                  00804ff0    00000018     JpegEncApp6678.pe66.obj (.const:xdc_runtime_GateNull_Object__PARAMS__C)
                  00805008    00000018     JpegEncApp6678.pe66.obj (.const:xdc_runtime_knl_GateThread_Object__PARAMS__C)
                  00805020    00000011     JpegEncApp6678.pe66.obj (.const:digtohex$52)
                  00805031    00000003     --HOLE--
                  00805034    0000000c     JpegEncApp6678.pe66.obj (.const:ti_sysbios_family_c66_Cache_initSize__C)
                  00805040    00000008     JpegEncApp6678.pe66.obj (.const:xdc_runtime_Startup_firstFxns__A)

.const.6   0    00805050    00000007     
                  00805050    00000007     rts6600_elf.lib : _scanfi.obj (.const:flit$1)

.const.7   0    00805060    00000006     
                  00805060    00000006     rts6600_elf.lib : _scanfi.obj (.const:barr$2)

.const.8   0    00805070    00000004     
                  00805070    00000004     JpegEncApp6678.pe66.obj (.const:ti_sdo_ipc_gates_GateHWSem_reservedMaskArr__A)

.const.9   0    00805080    00000004     
                  00805080    00000004     JpegEncApp6678.pe66.obj (.const:ti_sysbios_knl_Idle_funcList__A)

.stack     0    00805088    00002000     UNINITIALIZED
                  00805088    00000008     boot.ae66 : boot.oe66 (.stack)
                  00805090    00001ff8     --HOLE--

.fardata.1 
*          0    00807090    000016f8     
                  00807090    00000800     JpegEncApp6678.pe66.obj (.fardata:ti_sdo_ipc_GateMP_Module_State_0_remoteCustom1Gates__A)
                  00807890    000002f0     JpegEncApp6678.pe66.obj (.fardata)
                  00807b80    000001e0     rts6600_elf.lib : defs.obj (.fardata:_ftable)
                  00807d60    00000180     JpegEncApp6678.pe66.obj (.fardata:ti_sysbios_timers_timer64_Timer_Module_State_0_device__A)
                  00807ee0    000000e0     JpegEncApp6678.pe66.obj (.fardata:ti_sdo_utils_NameServer_Object__table__V)
                  00807fc0    000000b8     jpgealg_ti.le66 (.fardata:dmjpgegem_ti_ialg.oc)
                  00808078    00000008     rts6600_elf.lib : _lock.obj (.fardata)
                  00808080    000000a0                     : lowlev.obj (.fardata:_stream)
                  00808120    00000090     JpegEncApp6678.pe66.obj (.fardata:ti_sdo_ipc_SharedRegion_Module_State_0_regions__A)
                  008081b0    00000080     jpgealg_ti.le66 (.fardata:jpgenc_zigzag_scanorder:jpegtab.oc)
                  00808230    00000080     JpegEncApp6678.pe66.obj (.fardata:ti_sdo_ipc_GateMP_Module_State_0_remoteSystemGates__A)
                  008082b0    00000080     JpegEncApp6678.pe66.obj (.fardata:ti_sysbios_knl_Swi_Module_State_0_readyQ__A)
                  00808330    00000080     JpegEncApp6678.pe66.obj (.fardata:ti_sysbios_knl_Task_Module_State_0_readyQ__A)
                  008083b0    00000080     JpegEncApp6678.pe66.obj (.fardata:ti_sysbios_timers_timer64_Timer_Module_State_0_gctrl__A)
                  00808430    00000080     JpegEncApp6678.pe66.obj (.fardata:ti_sysbios_timers_timer64_Timer_Module_State_0_handles__A)
                  008084b0    00000080     JpegEncApp6678.pe66.obj (.fardata:ti_sysbios_timers_timer64_Timer_Module_State_0_intFreqs__A)
                  00808530    00000078     rts6600_elf.lib : lowlev.obj (.fardata:_device)
                  008085a8    00000004                     : defs.obj (.fardata)
                  008085ac    00000004                     : dtor_list.obj (.fardata)
                  008085b0    00000068     TestAppEncoder.obj (.fardata:sTokenMap)
                  00808618    00000004     rts6600_elf.lib : errno.obj (.fardata)
                  0080861c    00000004                     : fopen.obj (.fardata)
                  00808620    0000004c     JpegEncApp6678.pe66.obj (.fardata:ti_sysbios_timers_timer64_Timer_Object__table__V)
                  0080866c    00000004     rts6600_elf.lib : lowlev.obj (.fardata)
                  00808670    00000044     JpegEncApp6678.pe66.obj (.fardata:ti_sysbios_knl_Task_Object__table__V)
                  008086b4    0000000c     rts6600_elf.lib : exit.obj (.fardata)
                  008086c0    00000040     JpegEncApp6678.pe66.obj (.fardata:ti_sysbios_gates_GateMutex_Object__table__V)
                  00808700    00000030     JpegEncApp6678.pe66.obj (.fardata:ti_sysbios_knl_Swi_Object__table__V)
                  00808730    00000020     JpegEncApp6678.pe66.obj (.fardata:ti_sdo_ipc_MessageQ_Module_State_0_heaps__A)
                  00808750    00000020     JpegEncApp6678.pe66.obj (.fardata:xdc_runtime_System_Module_State_0_atexitHandlers__A)
                  00808770    00000018     JpegEncApp6678.pe66.obj (.fardata:ti_sysbios_family_c64p_Hwi_Object__table__V)

.fardata.2 
*          0    00808790    00000018     
                  00808790    00000018     JpegEncApp6678.pe66.obj (.fardata:ti_sysbios_gates_GateMutexPri_Object__table__V)

.fardata.3 
*          0    008087b0    00000014     
                  008087b0    00000014     JpegEncApp6678.pe66.obj (.fardata:ti_sdo_ipc_Ipc_Module_State_0_procEntry__A)

.fardata.4 
*          0    008087d0    00000014     
                  008087d0    00000014     JpegEncApp6678.pe66.obj (.fardata:ti_sysbios_heaps_HeapMem_Object__table__V)

.fardata.5 
*          0    008087f0    00000028     
                  008087f0    00000010     JpegEncApp6678.pe66.obj (.fardata:ti_sysbios_gates_GateAll_Object__table__V)
                  00808800    0000000c     JpegEncApp6678.pe66.obj (.fardata:ti_sysbios_gates_GateSwi_Object__table__V)
                  0080880c    00000004     --HOLE--
                  00808810    00000008     JpegEncApp6678.pe66.obj (.fardata:ti_sdo_ipc_MessageQ_Module_State_0_transports__A)

.fardata.6 
*          0    00808820    00000008     
                  00808820    00000008     JpegEncApp6678.pe66.obj (.fardata:ti_sysbios_hal_Hwi_Object__table__V)

.fardata.7 
*          0    00808830    00000008     
                  00808830    00000008     JpegEncApp6678.pe66.obj (.fardata:ti_sysbios_hal_Timer_Object__table__V)

.fardata.8 
*          0    00808840    00000004     
                  00808840    00000004     JpegEncApp6678.pe66.obj (.fardata:ti_sdo_ipc_GateMP_Module_State_0_remoteCustom2Gates__A)

.fardata.9 
*          0    00808850    00000004     
                  00808850    00000004     JpegEncApp6678.pe66.obj (.fardata:ti_sdo_ipc_Notify_Module_State_0_notifyHandles_0__A)

.fardata.10 
*          0    00808860    00000004     
                  00808860    00000004     JpegEncApp6678.pe66.obj (.fardata:ti_sdo_ipc_Notify_Module_State_0_notifyHandles__A)

.fardata.11 
*          0    00808870    00000004     
                  00808870    00000004     JpegEncApp6678.pe66.obj (.fardata:ti_sdo_ipc_transports_TransportShmSetup_Module_State_0_handles__A)

.fardata.12 
*          0    00808880    00000004     
                  00808880    00000004     JpegEncApp6678.pe66.obj (.fardata:xdc_runtime_GateNull_Object__table__V)

.taskStackSection 
*          0    00808888    00000800     UNINITIALIZED
                  00808888    00000800     JpegEncApp6678.pe66.obj (.taskStackSection)

.args      0    00809088    00000200     
                  00809088    00000200     --HOLE-- [fill = 0]

.switch    0    00809288    000001a4     
                  00809288    00000074     jpgealg_ti.le66 (.switch:DMJPGE_setDynamicParams:jpgegemAPI.oc)
                  008092fc    0000002c     jpgealg_ti.le66 (.switch:DMJPGE_initializeScan:jpgegemAPI.oc)
                  00809328    00000028     rts6600_elf.lib : _scanfi.obj (.switch:_sset_arg)
                  00809350    00000020     TestAppEncoder.obj (.switch:Initialize_original_buffer)
                  00809370    0000001c     jpgealg_ti.le66 (.switch:DMJPGE_TIGEM_xdmControl:dmjpgegem_ti_ialg.oc)
                  0080938c    0000001c     jpgealg_ti.le66 (.switch:DMJPGE_getCurrentIteration:jpgegemAPI.oc)
                  008093a8    0000001c     jpgealg_ti.le66 (.switch:DMJPGE_getTotalIterations:jpgegemAPI.oc)
                  008093c4    0000001c     jpgealg_ti.le66 (.switch:jpgeGenHeader:jpgeGenHeader.oc)
                  008093e0    0000001c     jpgealg_ti.le66 (.switch:set_Thumbnail_params:jpgethumbnail.oc)
                  008093fc    00000010     jpgealg_ti.le66 (.switch:DMJPGE_insertScanHeader:jpgegemAPI.oc)
                  0080940c    00000010     jpgealg_ti.le66 (.switch:DMJPGE_updateState:jpgegemAPI.oc)
                  0080941c    00000010     JpegEncApp6678.pe66.obj (.switch:ti_sdo_ipc_GateMP_Instance_finalize__F)

.cio       0    0080942c    00000120     UNINITIALIZED
                  0080942c    00000120     rts6600_elf.lib : trgmsg.obj (.cio)

.bss       0    00809550    00000030     UNINITIALIZED
                  00809550    00000030     TestAppEncoder.obj (.bss)

.neardata 
*          0    00809580    00000010     
                  00809580    00000008     TestAppEncoder.obj (.neardata)
                  00809588    00000008     alg_malloc.obj (.neardata)

.rodata    0    00809590    00000000     UNINITIALIZED

.cinit     0    00809590    000052e8     
                  00809590    00004231     (.cinit..const.1.load) [load image, compression = rle]
                  0080d7c1    00000003     --HOLE-- [fill = 0]
                  0080d7c4    0000088e     (.cinit..fardata.1.load) [load image, compression = rle]
                  0080e052    00000002     --HOLE-- [fill = 0]
                  0080e054    000004be     (.cinit..const.4.load) [load image, compression = rle]
                  0080e512    00000002     --HOLE-- [fill = 0]
                  0080e514    0000009d     (.cinit..const.2.load) [load image, compression = rle]
                  0080e5b1    00000003     --HOLE-- [fill = 0]
                  0080e5b4    00000059     (.cinit..const.5.load) [load image, compression = rle]
                  0080e60d    00000003     --HOLE-- [fill = 0]
                  0080e610    00000045     (.cinit..const.3.load) [load image, compression = rle]
                  0080e655    00000003     --HOLE-- [fill = 0]
                  0080e658    0000001a     (.cinit..fardata.5.load) [load image, compression = rle]
                  0080e672    00000002     --HOLE-- [fill = 0]
                  0080e674    00000018     (.cinit..fardata.4.load) [load image, compression = rle]
                  0080e68c    00000016     (.cinit..fardata.2.load) [load image, compression = rle]
                  0080e6a2    00000002     --HOLE-- [fill = 0]
                  0080e6a4    00000015     (.cinit..neardata.load) [load image, compression = rle]
                  0080e6b9    00000003     --HOLE-- [fill = 0]
                  0080e6bc    0000000f     (.cinit..fardata.3.load) [load image, compression = rle]
                  0080e6cb    00000001     --HOLE-- [fill = 0]
                  0080e6cc    0000000d     (.cinit..const.6.load) [load image, compression = rle]
                  0080e6d9    00000003     --HOLE-- [fill = 0]
                  0080e6dc    0000000d     (.cinit..fardata.6.load) [load image, compression = rle]
                  0080e6e9    00000003     --HOLE-- [fill = 0]
                  0080e6ec    0000000d     (.cinit..fardata.7.load) [load image, compression = rle]
                  0080e6f9    00000003     --HOLE-- [fill = 0]
                  0080e6fc    0000000c     (.cinit..const.7.load) [load image, compression = rle]
                  0080e708    0000000c     (__TI_handler_table)
                  0080e714    0000000a     (.cinit..const.9.load) [load image, compression = rle]
                  0080e71e    00000002     --HOLE-- [fill = 0]
                  0080e720    0000000a     (.cinit..fardata.10.load) [load image, compression = rle]
                  0080e72a    00000002     --HOLE-- [fill = 0]
                  0080e72c    0000000a     (.cinit..fardata.12.load) [load image, compression = rle]
                  0080e736    00000002     --HOLE-- [fill = 0]
                  0080e738    00000009     (.cinit..const.8.load) [load image, compression = rle]
                  0080e741    00000003     --HOLE-- [fill = 0]
                  0080e744    00000009     (.cinit..fardata.11.load) [load image, compression = rle]
                  0080e74d    00000003     --HOLE-- [fill = 0]
                  0080e750    00000009     (.cinit..fardata.8.load) [load image, compression = rle]
                  0080e759    00000003     --HOLE-- [fill = 0]
                  0080e75c    00000009     (.cinit..fardata.9.load) [load image, compression = rle]
                  0080e765    00000003     --HOLE-- [fill = 0]
                  0080e768    00000008     (.cinit..bitsData.load) [load image, compression = zero_init]
                  0080e770    00000008     (.cinit..bss.load) [load image, compression = zero_init]
                  0080e778    00000008     (.cinit..ccdData.load) [load image, compression = zero_init]
                  0080e780    00000008     (.cinit..far.load) [load image, compression = zero_init]
                  0080e788    00000008     (.cinit..ref_buffer.load) [load image, compression = zero_init]
                  0080e790    00000008     (.cinit..taskStackSection.load) [load image, compression = zero_init]
                  0080e798    000000e0     (__TI_cinit_table)

.text      0    0c000000    00023e40     
                  0c000000    00007da0     jpgealg_ti.le66 (.text:JPEGIENC_TI_cSect)
                  0c007da0    00000ea0     TestAppEncoder.obj (.text:EncodeTask)
                  0c008c40    00000c00     JpegEncApp6678.pe66.obj (.text:ti_sdo_ipc_GateMP_Instance_init__F)
                  0c009840    00000a80     JpegEncApp6678.pe66.obj (.text:xdc_runtime_System_doPrint__I)
                  0c00a2c0    00000940     rts6600_elf.lib : _scanfi.obj (.text:_scanfi)
                  0c00ac00    00000820     jpgealg_ti.le66 (.text:xdmControl:DMJPGE_TIGEM_xdmProcess:dmjpgegem_ti_ialg.oc)
                  0c00b420    00000700     JpegEncApp6678.pe66.obj (.text:ti_sysbios_family_c64p_Exception_handler__I)
                  0c00bb20    000006e0     rts6600_elf.lib : _scanfi.obj (.text:_sset_arg)
                  0c00c200    00000660     JpegEncApp6678.pe66.obj (.text:NameServer_add)
                  0c00c860    000005e0     alg_malloc.obj (.text:_ALG_allocMemory)
                  0c00ce40    000005c0     rts6600_elf.lib : divd.obj (.text:__c6xabi_divd)
                  0c00d400    000005c0                     : _printfi.obj (.text:_getarg_diouxp)
                  0c00d9c0    00000580     jpgealg_ti.le66 (.text:DMJPGE_TIGEM_xdmControl:dmjpgegem_ti_ialg.oc)
                  0c00df40    00000520     rts6600_elf.lib : strtod.obj (.text:strtod)
                  0c00e460    00000500                     : strtold.obj (.text:strtold)
                  0c00e960    000004c0                     : _scanfi.obj (.text:_sproc_int)
                  0c00ee20    00000480                     : _printfi.obj (.text:_setfield)
                  0c00f2a0    00000480                     : fwrite.obj (.text:fwrite)
                  0c00f720    00000460                     : _printfi.obj (.text:_printfi)
                  0c00fb80    00000460                     : strtoll.obj (.text:strtoll)
                  0c00ffe0    00000420     JpegEncApp6678.pe66.obj (.text:ti_sdo_ipc_GateMP_Instance_finalize__F)
                  0c010400    00000400     rts6600_elf.lib : strtoull.obj (.text:strtoull)
                  0c010800    00000400     JpegEncApp6678.pe66.obj (.text:ti_sdo_ipc_heaps_HeapMemMP_alloc__F)
                  0c010c00    000003e0     JpegEncApp6678.pe66.obj (.text:ti_sdo_ipc_heaps_HeapMemMP_Instance_init__F)
                  0c010fe0    000003c0     JpegEncApp6678.pe66.obj (.text:ti_sdo_ipc_gates_GatePeterson_Instance_init__F)
                  0c0113a0    000003a0     TestAppConfigParser.obj (.text:ParseContent)
                  0c011740    000003a0     rts6600_elf.lib : strtol.obj (.text:strtol)
                  0c011ae0    00000360     JpegEncApp6678.pe66.obj (.text:GateMP_sharedMemReq)
                  0c011e40    00000360     JpegEncApp6678.pe66.obj (.text:ti_sysbios_gates_GateMutexPri_enter__E)
                  0c0121a0    00000340     rts6600_elf.lib : _scanfi.obj (.text:_sget_conv)
                  0c0124e0    00000340     JpegEncApp6678.pe66.obj (.text:ti_sdo_ipc_GateMP_setRegion0Reserved__F)
                  0c012820    00000340     JpegEncApp6678.pe66.obj (.text:ti_sdo_ipc_heaps_HeapMemMP_free__F)
                  0c012b60    00000340     JpegEncApp6678.pe66.obj (.text:ti_sysbios_knl_Semaphore_pend__E)
                  0c012ea0    00000320     rts6600_elf.lib : fgets.obj (.text:_dofgets)
                  0c0131c0    00000300     jpgealg_ti.le66 (.text:DMJPGE_TIGEM_algInit:dmjpgegem_ti_ialg.oc)
                  0c0134c0    00000300     rts6600_elf.lib : fputs.obj (.text:fputs)
                  0c0137c0    00000300                     : strtoul.obj (.text:strtoul)
                  0c013ac0    00000300     JpegEncApp6678.pe66.obj (.text:ti_sysbios_knl_Task_Instance_finalize__F)
                  0c013dc0    00000300     JpegEncApp6678.pe66.obj (.text:ti_sysbios_timers_timer64_Timer_Module_startup__F)
                  0c0140c0    00000300     JpegEncApp6678.pe66.obj (.text:xdc_runtime_System_printfExtend__I)
                  0c0143c0    000002e0     rts6600_elf.lib : _printfi.obj (.text:_pproc_fwp)
                  0c0146a0    000002e0                     : _scanfi.obj (.text:_sproc_float)
                  0c014980    000002e0     JpegEncApp6678.pe66.obj (.text:ti_sdo_ipc_SharedRegion_start__F)
                  0c014c60    000002c0     JpegEncApp6678.pe66.obj (.text:GateMP_openByAddr)
                  0c014f20    000002c0     rts6600_elf.lib : _printfi.obj (.text:_pproc_fge)
                  0c0151e0    000002a0                     : _printfi.obj (.text:fcvt)
                  0c015480    000002a0                     : fread.obj (.text:fread)
                  0c015720    00000280     JpegEncApp6678.pe66.obj (.text:deviceConfig$19)
                  0c0159a0    00000280     rts6600_elf.lib : _printfi.obj (.text:ecvt)
                  0c015c20    00000280     JpegEncApp6678.pe66.obj (.text:ti_sdo_utils_NameServer_removeLocal__I)
                  0c015ea0    00000260     JpegEncApp6678.pe66.obj (.text:ti_sysbios_heaps_HeapMem_free__E)
                  0c016100    00000260     JpegEncApp6678.pe66.obj (.text:ti_sysbios_knl_Task_setPri__E)
                  0c016360    00000240     TestAppEncoder.obj (.text:Initialize_original_buffer)
                  0c0165a0    00000240     rts6600_elf.lib : imath64.obj (.text:__c6xabi_divull)
                  0c0167e0    00000240                     : _printfi.obj (.text:_pconv_e)
                  0c016a20    00000240                     : _printfi.obj (.text:_pproc_diouxp)
                  0c016c60    00000240     JpegEncApp6678.pe66.obj (.text:ti_sysbios_knl_Task_Instance_init__F)
                  0c016ea0    00000220     rts6600_elf.lib : _printfi.obj (.text:_pproc_str)
                  0c0170c0    00000220     JpegEncApp6678.pe66.obj (.text:ti_sdo_ipc_heaps_HeapMemMP_postInit__I)
                  0c0172e0    00000220     JpegEncApp6678.pe66.obj (.text:ti_sysbios_BIOS_startFunc__I)
                  0c017500    00000220     JpegEncApp6678.pe66.obj (.text:ti_sysbios_family_c64p_Exception_internalHandler__I)
                  0c017720    00000220     JpegEncApp6678.pe66.obj (.text:ti_sysbios_knl_Task_postInit__I)
                  0c017940    00000220     JpegEncApp6678.pe66.obj (.text:xdc_runtime_Core_createObject__I)
                  0c017b60    00000200     rts6600_elf.lib : _printfi.obj (.text:_pconv_g)
                  0c017d60    00000200     ti.sysbios.family.c64p.ae66 : Hwi_disp_always.oe66 (.text:_ti_sysbios_family_c64p_Hwi_dispatchAlways)
                  0c017f60    00000200     JpegEncApp6678.pe66.obj (.text:ti_sdo_ipc_GateMP_getFreeResource__I)
                  0c018160    000001e0     JpegEncApp6678.pe66.obj (.text:ti_sysbios_heaps_HeapMem_alloc__E)
                  0c018340    000001e0     JpegEncApp6678.pe66.obj (.text:ti_sysbios_knl_Swi_schedule__I)
                  0c018520    000001c0     JpegEncApp6678.pe66.obj (.text:HeapMemMP_sharedMemReq)
                  0c0186e0    000001c0     JpegEncApp6678.pe66.obj (.text:Ipc_start)
                  0c0188a0    000001c0     rts6600_elf.lib : _printfi.obj (.text:_mcpy)
                  0c018a60    000001c0                     : fopen.obj (.text:_openfile)
                  0c018c20    000001c0     JpegEncApp6678.pe66.obj (.text:ti_sdo_ipc_Notify_Instance_init__F)
                  0c018de0    000001c0     JpegEncApp6678.pe66.obj (.text:ti_sysbios_gates_GateMutexPri_leave__E)
                  0c018fa0    000001c0     JpegEncApp6678.pe66.obj (.text:ti_sysbios_knl_Task_checkStacks__E)
                  0c019160    000001c0     JpegEncApp6678.pe66.obj (.text:ti_sysbios_timers_timer64_Timer_setPeriodMicroSecs__E)
                  0c019320    000001c0     JpegEncApp6678.pe66.obj (.text:xdc_runtime_Startup_startMods__I)
                  0c0194e0    000001a0     rts6600_elf.lib : trgdrv.obj (.text:HOSTrename)
                  0c019680    000001a0                     : imath40.obj (.text:__c6xabi_divul)
                  0c019820    000001a0                     : _scanfi.obj (.text:_sproc_lb)
                  0c0199c0    000001a0                     : _scanfi.obj (.text:_sproc_str)
                  0c019b60    000001a0     JpegEncApp6678.pe66.obj (.text:ti_sdo_ipc_SharedRegion_reserveMemory__F)
                  0c019d00    000001a0     JpegEncApp6678.pe66.obj (.text:ti_sysbios_timers_timer64_Timer_start__E)
                  0c019ea0    000001a0     JpegEncApp6678.pe66.obj (.text:xdc_runtime_Text_putSite__F)
                  0c01a040    00000180     jpgealg_ti.le66 (.text:DMJPGE_TIGEM_algFree:dmjpgegem_ti_ialg.oc)
                  0c01a1c0    00000180     rts6600_elf.lib : copy_decompress_rle.obj (.text:__TI_decompress_rle_core)
                  0c01a340    00000180     JpegEncApp6678.pe66.obj (.text:block$41)
                  0c01a4c0    00000180     rts6600_elf.lib : lowlev.obj (.text:open)
                  0c01a640    00000180                     : setvbuf.obj (.text:setvbuf)
                  0c01a7c0    00000180     ti.sysbios.family.c64p.ae66 : Exception_asm.oe66 (.text)
                  0c01a940    00000180     JpegEncApp6678.pe66.obj (.text:ti_sdo_ipc_gates_GatePeterson_enter__F)
                  0c01aac0    00000180     JpegEncApp6678.pe66.obj (.text:xdc_runtime_Error_raiseX__F)
                  0c01ac40    00000160     boot.ae66 : autoinit.oe66 (.text:_auto_init_elf)
                  0c01ada0    00000160     JpegEncApp6678.pe66.obj (.text:ti_sdo_ipc_GateMP_start__F)
                  0c01af00    00000160     JpegEncApp6678.pe66.obj (.text:ti_sysbios_family_c64p_Hwi_dispatchC__I)
                  0c01b060    00000160     JpegEncApp6678.pe66.obj (.text:ti_sysbios_knl_Clock_Object__create__S)
                  0c01b1c0    00000160     JpegEncApp6678.pe66.obj (.text:ti_sysbios_knl_Task_exit__E)
                  0c01b320    00000160     JpegEncApp6678.pe66.obj (.text:xdc_runtime_Core_deleteObject__I)
                  0c01b480    00000160     JpegEncApp6678.pe66.obj (.text:xdc_runtime_Text_visitRope2__I)
                  0c01b5e0    00000140     JpegEncApp6678.pe66.obj (.text:HeapMemMP_create)
                  0c01b720    00000140     rts6600_elf.lib : _bufread.obj (.text:_buff_read)
                  0c01b860    00000140                     : sscanf.obj (.text:_chkmbc)
                  0c01b9a0    00000140                     : _printfi.obj (.text:_pproc_fflags)
                  0c01bae0    00000140                     : fputc.obj (.text:fputc)
                  0c01bc20    00000140                     : lowlev.obj (.text:getdevice)
                  0c01bd60    00000140     JpegEncApp6678.pe66.obj (.text:ti_sysbios_family_c64p_Hwi_Module_startup__F)
                  0c01bea0    00000140     JpegEncApp6678.pe66.obj (.text:ti_sysbios_family_c66_Cache_Module_startup__F)
                  0c01bfe0    00000120     TestAppEncoder.obj (.text:TestApp_ReadInputData)
                  0c01c100    00000120     rts6600_elf.lib : imath64.obj (.text:__c6xabi_divlli)
                  0c01c220    00000120                     : _printfi.obj (.text:_ltostr)
                  0c01c340    00000120                     : fopen.obj (.text:_search_fp)
                  0c01c460    00000120                     : _scanfi.obj (.text:_sget_scanset)
                  0c01c580    00000120                     : _io_perm.obj (.text:_wrt_ok)
                  0c01c6a0    00000120                     : fclose.obj (.text:fclose)
                  0c01c7c0    00000120     JpegEncApp6678.pe66.obj (.text:ti_sdo_ipc_heaps_HeapMemMP_Instance_finalize__F)
                  0c01c8e0    00000120     JpegEncApp6678.pe66.obj (.text:ti_sdo_ipc_heaps_HeapMemMP_getStats__F)
                  0c01ca00    00000120     JpegEncApp6678.pe66.obj (.text:ti_sysbios_knl_Clock_workFunc__E)
                  0c01cb20    00000120     JpegEncApp6678.pe66.obj (.text:ti_sysbios_knl_Task_schedule__I)
                  0c01cc40    00000120     JpegEncApp6678.pe66.obj (.text:xdc_runtime_SysMin_flush__F)
                  0c01cd60    00000100     rts6600_elf.lib : trgdrv.obj (.text:HOSTlseek)
                  0c01ce60    00000100     alg_create.obj (.text:create:ALG_create)
                  0c01cf60    00000100     rts6600_elf.lib : fflush.obj (.text:fflush)
                  0c01d060    00000100     JpegEncApp6678.pe66.obj (.text:ti_sdo_ipc_gates_GateHWSem_Module_startup__F)
                  0c01d160    00000100     JpegEncApp6678.pe66.obj (.text:ti_sdo_ipc_gates_GateHWSem_enter__F)
                  0c01d260    00000100     JpegEncApp6678.pe66.obj (.text:ti_sdo_ipc_gates_GatePeterson_Object__create__S)
                  0c01d360    00000100     JpegEncApp6678.pe66.obj (.text:ti_sdo_ipc_heaps_HeapMemMP_Object__create__S)
                  0c01d460    00000100     JpegEncApp6678.pe66.obj (.text:ti_sdo_utils_NameServer_Module_startup__F)
                  0c01d560    00000100     JpegEncApp6678.pe66.obj (.text:ti_sysbios_gates_GateAll_leave__E)
                  0c01d660    00000100     JpegEncApp6678.pe66.obj (.text:ti_sysbios_heaps_HeapMem_Object__create__S)
                  0c01d760    00000100     JpegEncApp6678.pe66.obj (.text:ti_sysbios_knl_Semaphore_post__E)
                  0c01d860    00000100     JpegEncApp6678.pe66.obj (.text:ti_sysbios_knl_Swi_restoreHwi__E)
                  0c01d960    00000100     JpegEncApp6678.pe66.obj (.text:ti_sysbios_knl_Task_Object__create__S)
                  0c01da60    00000100     JpegEncApp6678.pe66.obj (.text:ti_sysbios_knl_Task_startup__E)
                  0c01db60    00000100     JpegEncApp6678.pe66.obj (.text:xdc_runtime_Memory_alloc__F)
                  0c01dc60    00000100     JpegEncApp6678.pe66.obj (.text:xdc_runtime_Text_putMod__F)
                  0c01dd60    00000100     JpegEncApp6678.pe66.obj (.text:xdc_runtime_knl_GateThread_Object__create__S)
                  0c01de60    000000e0     JpegEncApp6678.pe66.obj (.text:GateMP_close)
                  0c01df40    000000e0     rts6600_elf.lib : trgdrv.obj (.text:HOSTopen)
                  0c01e020    000000e0                     : divi.obj (.text:__divi)
                  0c01e100    000000e0                     : _printfi.obj (.text:_div)
                  0c01e1e0    000000e0                     : atoi.obj (.text:atoi)
                  0c01e2c0    000000e0                     : lowlev.obj (.text:close)
                  0c01e3a0    000000e0                     : copy_zero_init.obj (.text:decompress:ZI:__TI_zero_init)
                  0c01e480    000000e0                     : exit.obj (.text:exit)
                  0c01e560    000000e0     JpegEncApp6678.pe66.obj (.text:initDevice$19)
                  0c01e640    000000e0     rts6600_elf.lib : ltoa.obj (.text:ltoa)
                  0c01e720    000000e0     JpegEncApp6678.pe66.obj (.text:memalign)
                  0c01e800    000000e0     rts6600_elf.lib : memset.obj (.text:memset)
                  0c01e8e0    000000e0     JpegEncApp6678.pe66.obj (.text:ti_sdo_ipc_GateMP_Object__create__S)
                  0c01e9c0    000000e0     JpegEncApp6678.pe66.obj (.text:ti_sdo_ipc_GateMP_createLocal__F)
                  0c01eaa0    000000e0     JpegEncApp6678.pe66.obj (.text:ti_sdo_ipc_gates_GateHWSem_Object__create__S)
                  0c01eb80    000000e0     JpegEncApp6678.pe66.obj (.text:ti_sysbios_gates_GateMutex_enter__E)
                  0c01ec60    000000e0     JpegEncApp6678.pe66.obj (.text:ti_sysbios_gates_GateSwi_leave__E)
                  0c01ed40    000000e0     JpegEncApp6678.pe66.obj (.text:ti_sysbios_knl_Semaphore_Object__create__S)
                  0c01ee20    000000e0     JpegEncApp6678.pe66.obj (.text:ti_sysbios_timers_timer64_Timer_stop__E)
                  0c01ef00    000000c0     jpgealg_ti.le66 (.text:DMJPGE_TIGEM_algAlloc:dmjpgegem_ti_ialg.oc)
                  0c01efc0    000000c0     JpegEncApp6678.pe66.obj (.text:GateMP_Params_init)
                  0c01f080    000000c0     rts6600_elf.lib : trgdrv.obj (.text:HOSTread)
                  0c01f140    000000c0                     : trgdrv.obj (.text:HOSTunlink)
                  0c01f200    000000c0                     : trgdrv.obj (.text:HOSTwrite)
                  0c01f2c0    000000c0     JpegEncApp6678.pe66.obj (.text:HeapMemMP_Params_init)
                  0c01f380    000000c0     TestAppEncoder.obj (.text:TestApp_WriteOutputData)
                  0c01f440    000000c0     alg_malloc.obj (.text:_ALG_freeMemory)
                  0c01f500    000000c0     rts6600_elf.lib : dtor_list.obj (.text:__cxa_finalize)
                  0c01f5c0    000000c0                     : divu.obj (.text:__divu)
                  0c01f680    000000c0                     : fopen.obj (.text:_cleanup)
                  0c01f740    000000c0                     : fflush.obj (.text:_doflush)
                  0c01f800    000000c0                     : _io_perm.obj (.text:_rd_ok)
                  0c01f8c0    000000c0     alg_create.obj (.text:delete:ALG_delete)
                  0c01f980    000000c0     rts6600_elf.lib : fseek.obj (.text:fseek)
                  0c01fa40    000000c0                     : lowlev.obj (.text:lseek)
                  0c01fb00    000000c0                     : lowlev.obj (.text:read)
                  0c01fbc0    000000c0     JpegEncApp6678.pe66.obj (.text:ti_sdo_ipc_MessageQ_Module_startup__F)
                  0c01fc80    000000c0     JpegEncApp6678.pe66.obj (.text:ti_sysbios_family_c66_Cache_setMar__E)
                  0c01fd40    000000c0     JpegEncApp6678.pe66.obj (.text:ti_sysbios_heaps_HeapMem_getStats__E)
                  0c01fe00    000000c0     JpegEncApp6678.pe66.obj (.text:ti_sysbios_knl_Swi_run__I)
                  0c01fec0    000000c0     rts6600_elf.lib : lowlev.obj (.text:write)
                  0c01ff80    000000a0     TestAppConfigParser.obj (.text:GetConfigFileContent)
                  0c020020    000000a0     rts6600_elf.lib : trgdrv.obj (.text:HOSTclose)
                  0c0200c0    000000a0     JpegEncApp6678.pe66.obj (.text:SharedRegion_getCacheLineSize)
                  0c020160    000000a0     JpegEncApp6678.pe66.obj (.text:SharedRegion_getHeap)
                  0c020200    000000a0     JpegEncApp6678.pe66.obj (.text:SharedRegion_getId)
                  0c0202a0    000000a0     JpegEncApp6678.pe66.obj (.text:SharedRegion_isCacheEnabled)
                  0c020340    000000a0     TestAppEncoder.obj (.text:TestApp_CompareOutputData)
                  0c0203e0    000000a0     rts6600_elf.lib : remu.obj (.text:__remu)
                  0c020480    000000a0     boot.ae66 : boot.oe66 (.text:_c_int00)
                  0c020520    000000a0     rts6600_elf.lib : _printfi.obj (.text:_ecpy)
                  0c0205c0    000000a0                     : _printfi.obj (.text:_fcpy)
                  0c020660    000000a0                     : _printfi.obj (.text:_pconv_f)
                  0c020700    000000a0                     : lowlev.obj (.text:finddevice)
                  0c0207a0    000000a0                     : ftell.obj (.text:ftell)
                  0c020840    000000a0                     : memcpy64.obj (.text:memcpy)
                  0c0208e0    000000a0                     : lowlev.obj (.text:tabinit)
                  0c020980    000000a0     JpegEncApp6678.pe66.obj (.text:ti_sdo_ipc_GateMP_getRegion0ReservedSize__F)
                  0c020a20    000000a0     JpegEncApp6678.pe66.obj (.text:ti_sdo_ipc_Notify_Object__create__S)
                  0c020ac0    000000a0     JpegEncApp6678.pe66.obj (.text:ti_sdo_ipc_gates_GatePeterson_leave__F)
                  0c020b60    000000a0     JpegEncApp6678.pe66.obj (.text:ti_sysbios_BIOS_exitFunc__I)
                  0c020c00    000000a0     JpegEncApp6678.pe66.obj (.text:ti_sysbios_gates_GateMutexPri_Object__create__S)
                  0c020ca0    000000a0     JpegEncApp6678.pe66.obj (.text:ti_sysbios_gates_GateMutex_Object__create__S)
                  0c020d40    000000a0     JpegEncApp6678.pe66.obj (.text:ti_sysbios_gates_GateSwi_enter__E)
                  0c020de0    000000a0     JpegEncApp6678.pe66.obj (.text:ti_sysbios_knl_Clock_Instance_finalize__F)
                  0c020e80    000000a0     JpegEncApp6678.pe66.obj (.text:ti_sysbios_knl_Task_Params__init__S)
                  0c020f20    000000a0     JpegEncApp6678.pe66.obj (.text:ti_sysbios_xdcruntime_GateThreadSupport_Object__create__S)
                  0c020fc0    000000a0     JpegEncApp6678.pe66.obj (.text:xdc_runtime_Error_print__F)
                  0c021060    000000a0     JpegEncApp6678.pe66.obj (.text:xdc_runtime_System_abort__F)
                  0c021100    000000a0     JpegEncApp6678.pe66.obj (.text:xdc_runtime_Text_xprintf__I)
                  0c0211a0    00000080     JpegEncApp6678.pe66.obj (.text:GateMP_enter)
                  0c021220    00000080     JpegEncApp6678.pe66.obj (.text:GateMP_leave)
                  0c0212a0    00000080     TestAppConfigParser.obj (.text:ParameterNameToMapIndex)
                  0c021320    00000080     TestAppEncoder.obj (.text:TestApp_EnableCache)
                  0c0213a0    00000080     rts6600_elf.lib : dtor_list.obj (.text:_Z11__TI_atexitPFYvPvES_S_)
                  0c021420    00000080                     : llshift.obj (.text:__c6xabi_llshl)
                  0c0214a0    00000080     ti.sysbios.family.c62.ae66 : TaskSupport_asm.oe66 (.text:_ti_sysbios_family_c62_TaskSupport_swap__E)
                  0c021520    00000080     rts6600_elf.lib : fprintf.obj (.text:fprintf)
                  0c0215a0    00000080     JpegEncApp6678.pe66.obj (.text:malloc)
                  0c021620    00000080     rts6600_elf.lib : printf.obj (.text:printf)
                  0c0216a0    00000080                     : trgmsg.obj (.text:readmsg)
                  0c021720    00000080                     : strncpy.obj (.text:strncpy)
                  0c0217a0    00000080     JpegEncApp6678.pe66.obj (.text:ti_sdo_ipc_Notify_Module_startup__F)
                  0c021820    00000080     JpegEncApp6678.pe66.obj (.text:ti_sysbios_family_c66_Cache_wbInvAll__E)
                  0c0218a0    00000080     JpegEncApp6678.pe66.obj (.text:ti_sysbios_gates_GateAll_Object__create__S)
                  0c021920    00000080     JpegEncApp6678.pe66.obj (.text:ti_sysbios_hal_Hwi_checkStack:ti_sysbios_hal_Hwi_checkStack)
                  0c0219a0    00000080     JpegEncApp6678.pe66.obj (.text:ti_sysbios_knl_Idle_loop__E)
                  0c021a20    00000080     JpegEncApp6678.pe66.obj (.text:ti_sysbios_knl_Semaphore_pendTimeout__I)
                  0c021aa0    00000080     JpegEncApp6678.pe66.obj (.text:ti_sysbios_knl_Swi_post__E)
                  0c021b20    00000080     JpegEncApp6678.pe66.obj (.text:ti_sysbios_knl_Task_unblockI__E)
                  0c021ba0    00000080     rts6600_elf.lib : lowlev.obj (.text:unlink)
                  0c021c20    00000080     JpegEncApp6678.pe66.obj (.text:xdc_runtime_Assert_raise__I)
                  0c021ca0    00000080     JpegEncApp6678.pe66.obj (.text:xdc_runtime_Startup_exec__F)
                  0c021d20    00000080     JpegEncApp6678.pe66.obj (.text:xdc_runtime_System_rtsExit__I)
                  0c021da0    00000080     JpegEncApp6678.pe66.obj (.text:xdc_runtime_Text_printVisFxn__I)
                  0c021e20    00000080     JpegEncApp6678.pe66.obj (.text:xdc_runtime_knl_GateThread_Instance_finalize__F)
                  0c021ea0    00000060     rts6600_elf.lib : frcmpyd_div.obj (.text:__c6xabi_frcmpyd_div)
                  0c021f00    00000060                     : llshift.obj (.text:__c6xabi_llshru)
                  0c021f60    00000060                     : imath64.obj (.text:__c6xabi_remull)
                  0c021fc0    00000060                     : imath64.obj (.text:_subcull)
                  0c022020    00000060                     : fopen.obj (.text:fopen)
                  0c022080    00000060                     : memccpy.obj (.text:memccpy)
                  0c0220e0    00000060                     : memcmp.obj (.text:memcmp)
                  0c022140    00000060     JpegEncApp6678.pe66.obj (.text:rtsLock$42)
                  0c0221a0    00000060     rts6600_elf.lib : sscanf.obj (.text:sscanf)
                  0c022200    00000060     JpegEncApp6678.pe66.obj (.text:ti_sdo_ipc_gates_GateHWSem_Object__delete__S)
                  0c022260    00000060     JpegEncApp6678.pe66.obj (.text:ti_sdo_ipc_gates_GateMPSupportNull_Object__create__S)
                  0c0222c0    00000060     JpegEncApp6678.pe66.obj (.text:ti_sdo_ipc_gates_GateMPSupportNull_Object__delete__S)
                  0c022320    00000060     JpegEncApp6678.pe66.obj (.text:ti_sdo_ipc_gates_GatePeterson_Instance_finalize__F)
                  0c022380    00000060     JpegEncApp6678.pe66.obj (.text:ti_sdo_ipc_gates_GatePeterson_Object__delete__S)
                  0c0223e0    00000060     JpegEncApp6678.pe66.obj (.text:ti_sdo_ipc_gates_GatePeterson_sharedMemReq__F)
                  0c022440    00000060     JpegEncApp6678.pe66.obj (.text:ti_sdo_ipc_heaps_HeapMemMP_Object__delete__S)
                  0c0224a0    00000060     JpegEncApp6678.pe66.obj (.text:ti_sdo_utils_List_Object__create__S)
                  0c022500    00000060     JpegEncApp6678.pe66.obj (.text:ti_sysbios_family_c64p_Exception_Module_startup__F)
                  0c022560    00000060     JpegEncApp6678.pe66.obj (.text:ti_sysbios_family_c66_Cache_setSize__E)
                  0c0225c0    00000060     JpegEncApp6678.pe66.obj (.text:ti_sysbios_gates_GateAll_Object__delete__S)
                  0c022620    00000060     JpegEncApp6678.pe66.obj (.text:ti_sysbios_gates_GateAll_enter__E)
                  0c022680    00000060     JpegEncApp6678.pe66.obj (.text:ti_sysbios_gates_GateMutexPri_Object__delete__S)
                  0c0226e0    00000060     JpegEncApp6678.pe66.obj (.text:ti_sysbios_gates_GateMutex_Object__delete__S)
                  0c022740    00000060     JpegEncApp6678.pe66.obj (.text:ti_sysbios_gates_GateSwi_Object__create__S)
                  0c0227a0    00000060     JpegEncApp6678.pe66.obj (.text:ti_sysbios_gates_GateSwi_Object__delete__S)
                  0c022800    00000060     JpegEncApp6678.pe66.obj (.text:ti_sysbios_hal_Hwi_initStack:ti_sysbios_hal_Hwi_initStack)
                  0c022860    00000060     JpegEncApp6678.pe66.obj (.text:ti_sysbios_heaps_HeapMem_Object__delete__S)
                  0c0228c0    00000060     JpegEncApp6678.pe66.obj (.text:ti_sysbios_knl_Clock_doTick__I)
                  0c022920    00000060     JpegEncApp6678.pe66.obj (.text:ti_sysbios_knl_Queue_Object__create__S)
                  0c022980    00000060     JpegEncApp6678.pe66.obj (.text:ti_sysbios_knl_Task_Module_startup__F)
                  0c0229e0    00000060     JpegEncApp6678.pe66.obj (.text:ti_sysbios_knl_Task_allBlockedFunction__I)
                  0c022a40    00000060     JpegEncApp6678.pe66.obj (.text:ti_sysbios_knl_Task_enter__I)
                  0c022aa0    00000060     rts6600_elf.lib : trgmsg.obj (.text:writemsg)
                  0c022b00    00000060     JpegEncApp6678.pe66.obj (.text:xdc_runtime_GateNull_Object__create__S)
                  0c022b60    00000060     JpegEncApp6678.pe66.obj (.text:xdc_runtime_GateNull_Object__delete__S)
                  0c022bc0    00000060     JpegEncApp6678.pe66.obj (.text:xdc_runtime_Memory_calloc__F)
                  0c022c20    00000060     JpegEncApp6678.pe66.obj (.text:xdc_runtime_SysMin_putch__F)
                  0c022c80    00000060     JpegEncApp6678.pe66.obj (.text:xdc_runtime_System_atexit__F)
                  0c022ce0    00000060     JpegEncApp6678.pe66.obj (.text:xdc_runtime_knl_GateThread_Object__delete__S)
                  0c022d40    00000040     rts6600_elf.lib : isinf.obj (.text:__c6xabi_isinf)
                  0c022d80    00000040                     : _printfi.obj (.text:__c6xabi_isnan)
                  0c022dc0    00000040                     : args_main.obj (.text:_args_main)
                  0c022e00    00000040     ti.sysbios.family.c62.ae66 : TaskSupport_asm.oe66 (.text:_ti_sysbios_family_c62_TaskSupport_buildTaskStack)
                  0c022e40    00000040     ti.sysbios.family.c64p.ae66 : Hwi_asm_switch.oe66 (.text:_ti_sysbios_family_xxx_Hwi_switchToIsrStack)
                  0c022e80    00000040     JpegEncApp6678.pe66.obj (.text:free)
                  0c022ec0    00000040     rts6600_elf.lib : abs.obj (.text:llabs)
                  0c022f00    00000040     TestAppEncoder.obj (.text:main)
                  0c022f40    00000040     TestAppConfigParser.obj (.text:readparamfile)
                  0c022f80    00000040     JpegEncApp6678.pe66.obj (.text:rtsUnlock$42)
                  0c022fc0    00000040     rts6600_elf.lib : strcmp.obj (.text:strcmp)
                  0c023000    00000040                     : strlen.obj (.text:strlen)
                  0c023040    00000040     JpegEncApp6678.pe66.obj (.text:ti_sdo_ipc_gates_GateHWSem_Handle__label__S)
                  0c023080    00000040     JpegEncApp6678.pe66.obj (.text:ti_sdo_ipc_gates_GateHWSem_leave__F)
                  0c0230c0    00000040     JpegEncApp6678.pe66.obj (.text:ti_sdo_ipc_gates_GateMPSupportNull_Handle__label__S)
                  0c023100    00000040     JpegEncApp6678.pe66.obj (.text:ti_sdo_ipc_gates_GateMPSupportNull_enter__F)
                  0c023140    00000040     JpegEncApp6678.pe66.obj (.text:ti_sdo_ipc_gates_GatePeterson_Handle__label__S)
                  0c023180    00000040     JpegEncApp6678.pe66.obj (.text:ti_sdo_ipc_heaps_HeapMemMP_Handle__label__S)
                  0c0231c0    00000040     JpegEncApp6678.pe66.obj (.text:ti_sysbios_gates_GateAll_Handle__label__S)
                  0c023200    00000040     JpegEncApp6678.pe66.obj (.text:ti_sysbios_gates_GateMutexPri_Handle__label__S)
                  0c023240    00000040     JpegEncApp6678.pe66.obj (.text:ti_sysbios_gates_GateMutexPri_Instance_finalize__F)
                  0c023280    00000040     JpegEncApp6678.pe66.obj (.text:ti_sysbios_gates_GateMutex_Handle__label__S)
                  0c0232c0    00000040     JpegEncApp6678.pe66.obj (.text:ti_sysbios_gates_GateMutex_Instance_finalize__F)
                  0c023300    00000040     JpegEncApp6678.pe66.obj (.text:ti_sysbios_gates_GateSwi_Handle__label__S)
                  0c023340    00000040     JpegEncApp6678.pe66.obj (.text:ti_sysbios_hal_Hwi_Module_startup__F)
                  0c023380    00000040     JpegEncApp6678.pe66.obj (.text:ti_sysbios_hal_Timer_Module_startup__F)
                  0c0233c0    00000040     JpegEncApp6678.pe66.obj (.text:ti_sysbios_heaps_HeapMem_Handle__label__S)
                  0c023400    00000040     JpegEncApp6678.pe66.obj (.text:ti_sysbios_heaps_HeapMem_init__I)
                  0c023440    00000040     JpegEncApp6678.pe66.obj (.text:ti_sysbios_knl_Clock_Module_startup__F)
                  0c023480    00000040     JpegEncApp6678.pe66.obj (.text:ti_sysbios_knl_Semaphore_Instance_finalize__F)
                  0c0234c0    00000040     TestAppEncoder.obj (.text:ti_sysbios_knl_Task_Params_init)
                  0c023500    00000040     TestAppEncoder.obj (.text:ti_sysbios_knl_Task_create)
                  0c023540    00000040     JpegEncApp6678.pe66.obj (.text:ti_sysbios_xdcruntime_GateThreadSupport_Instance_finalize__F)
                  0c023580    00000040     tsc_h.obj (.text)
                  0c0235c0    00000040     JpegEncApp6678.pe66.obj (.text:xdc_runtime_GateNull_Handle__label__S)
                  0c023600    00000040     JpegEncApp6678.pe66.obj (.text:xdc_runtime_Memory_free__F)
                  0c023640    00000040     JpegEncApp6678.pe66.obj (.text:xdc_runtime_SysMin_Module_startup__F)
                  0c023680    00000040     JpegEncApp6678.pe66.obj (.text:xdc_runtime_System_aprintf__E)
                  0c0236c0    00000040     JpegEncApp6678.pe66.obj (.text:xdc_runtime_System_printf__E)
                  0c023700    00000040     JpegEncApp6678.pe66.obj (.text:xdc_runtime_knl_GateThread_Handle__label__S)
                  0c023740    00000020     jpgealg_ti.le66 (.text:DMJPGE_TIGEM_activate:dmjpgegem_ti_ialg.oc)
                  0c023760    00000020     jpgealg_ti.le66 (.text:DMJPGE_TIGEM_algNumAlloc:dmjpgegem_ti_ialg.oc)
                  0c023780    00000020     jpgealg_ti.le66 (.text:DMJPGE_TIGEM_deactivate:dmjpgegem_ti_ialg.oc)
                  0c0237a0    00000020     TestAppEncoder.obj (.text:TestApp_SetDynamicParams)
                  0c0237c0    00000020     TestAppEncoder.obj (.text:TestApp_SetInitParams)
                  0c0237e0    00000020     rts6600_elf.lib : negll.obj (.text:__c6xabi_negll)
                  0c023800    00000020                     : dtor_list.obj (.text:__cxa_ia64_exit)
                  0c023820    00000020     JpegEncApp6678.pe66.obj (.text:__xdc__init)
                  0c023840    00000020     rts6600_elf.lib : sscanf.obj (.text:_inpchar)
                  0c023860    00000020                     : _lock.obj (.text:_nop)
                  0c023880    00000020                     : fprintf.obj (.text:_outc)
                  0c0238a0    00000020                     : printf.obj (.text:_outc)
                  0c0238c0    00000020                     : fprintf.obj (.text:_outs)
                  0c0238e0    00000020                     : printf.obj (.text:_outs)
                  0c023900    00000020                     : _lock.obj (.text:_register_lock)
                  0c023920    00000020                     : _lock.obj (.text:_register_unlock)
                  0c023940    00000020     ti.sysbios.family.c62.ae66 : TaskSupport_asm.oe66 (.text:_ti_sysbios_family_c62_TaskSupport_glue)
                  0c023960    00000020     ti.sysbios.family.c64p.ae66 : Hwi_asm_switch.oe66 (.text:_ti_sysbios_family_xxx_Hwi_switchToTaskStack)
                  0c023980    00000020     rts6600_elf.lib : sscanf.obj (.text:_uninpchar)
                  0c0239a0    00000020                     : exit.obj (.text:abort)
                  0c0239c0    00000020                     : dtor_list.obj (.text:atexit)
                  0c0239e0    00000020                     : copy_decompress_none.obj (.text:decompress:none:__TI_decompress_none)
                  0c023a00    00000020                     : copy_decompress_rle.obj (.text:decompress:rle24:__TI_decompress_rle24)
                  0c023a20    00000020                     : feof.obj (.text:feof)
                  0c023a40    00000020                     : fgets.obj (.text:fgets)
                  0c023a60    00000020     JpegEncApp6678.pe66.obj (.text:ti_sdo_ipc_gates_GateHWSem_getReservedMask__F)
                  0c023a80    00000020     JpegEncApp6678.pe66.obj (.text:ti_sdo_ipc_gates_GateHWSem_query__F)
                  0c023aa0    00000020     JpegEncApp6678.pe66.obj (.text:ti_sdo_ipc_gates_GateHWSem_sharedMemReq__F)
                  0c023ac0    00000020     JpegEncApp6678.pe66.obj (.text:ti_sdo_ipc_gates_GateMPSupportNull_getReservedMask__F)
                  0c023ae0    00000020     JpegEncApp6678.pe66.obj (.text:ti_sdo_ipc_gates_GateMPSupportNull_leave__F)
                  0c023b00    00000020     JpegEncApp6678.pe66.obj (.text:ti_sdo_ipc_gates_GateMPSupportNull_query__F)
                  0c023b20    00000020     JpegEncApp6678.pe66.obj (.text:ti_sdo_ipc_gates_GateMPSupportNull_sharedMemReq__F)
                  0c023b40    00000020     JpegEncApp6678.pe66.obj (.text:ti_sdo_ipc_gates_GatePeterson_getReservedMask__F)
                  0c023b60    00000020     JpegEncApp6678.pe66.obj (.text:ti_sdo_ipc_gates_GatePeterson_query__F)
                  0c023b80    00000020     JpegEncApp6678.pe66.obj (.text:ti_sdo_ipc_heaps_HeapMemMP_isBlocking__F)
                  0c023ba0    00000020     JpegEncApp6678.pe66.obj (.text:ti_sysbios_BIOS_start__E)
                  0c023bc0    00000020     JpegEncApp6678.pe66.obj (.text:ti_sysbios_family_c66_Cache_getMar__E)
                  0c023be0    00000020     JpegEncApp6678.pe66.obj (.text:ti_sysbios_family_c66_Cache_wbInv__E)
                  0c023c00    00000020     JpegEncApp6678.pe66.obj (.text:ti_sysbios_gates_GateAll_query__F)
                  0c023c20    00000020     JpegEncApp6678.pe66.obj (.text:ti_sysbios_gates_GateMutexPri_query__F)
                  0c023c40    00000020     JpegEncApp6678.pe66.obj (.text:ti_sysbios_gates_GateMutex_leave__E)
                  0c023c60    00000020     JpegEncApp6678.pe66.obj (.text:ti_sysbios_gates_GateMutex_query__F)
                  0c023c80    00000020     JpegEncApp6678.pe66.obj (.text:ti_sysbios_gates_GateSwi_query__F)
                  0c023ca0    00000020     JpegEncApp6678.pe66.obj (.text:ti_sysbios_heaps_HeapMem_isBlocking__E)
                  0c023cc0    00000020     JpegEncApp6678.pe66.obj (.text:ti_sysbios_knl_Swi_Module_startup__F)
                  0c023ce0    00000020     JpegEncApp6678.pe66.obj (.text:xdc_runtime_GateNull_enter__F)
                  0c023d00    00000020     JpegEncApp6678.pe66.obj (.text:xdc_runtime_GateNull_leave__F)
                  0c023d20    00000020     JpegEncApp6678.pe66.obj (.text:xdc_runtime_GateNull_query__F)
                  0c023d40    00000020     JpegEncApp6678.pe66.obj (.text:xdc_runtime_IGateProvider_leave$5)
                  0c023d60    00000020     JpegEncApp6678.pe66.obj (.text:xdc_runtime_Startup_exec__I)
                  0c023d80    00000020     JpegEncApp6678.pe66.obj (.text:xdc_runtime_Startup_reset__I)
                  0c023da0    00000020     JpegEncApp6678.pe66.obj (.text:xdc_runtime_System_Module_startup__F)
                  0c023dc0    00000020     JpegEncApp6678.pe66.obj (.text:xdc_runtime_System_exit__F)
                  0c023de0    00000020     JpegEncApp6678.pe66.obj (.text:xdc_runtime_Text_visitRope__I)
                  0c023e00    00000020     JpegEncApp6678.pe66.obj (.text:xdc_runtime_knl_GateThread_enter__F)
                  0c023e20    00000020     JpegEncApp6678.pe66.obj (.text:xdc_runtime_knl_GateThread_leave__F)

.vecs      0    0c024000    00000200     
                  0c024000    00000200     JpegEncApp6678.pe66.obj (.vecs)

.far       0    80000000    01f166e8     UNINITIALIZED
                  80000000    01f0f420     JpegEncApp6678.pe66.obj (.far)
                  81f0f420    00004e20     TestAppConfigParser.obj (.far)
                  81f14240    00002000     alg_malloc.obj (.far)
                  81f16240    00000290     TestAppEncoder.obj (.far)
                  81f164d0    00000140     rts6600_elf.lib : defs.obj (.far)
                  81f16610    000000d8                     : trgdrv.obj (.far)

.ccdData   0    81f166f0    00384000     UNINITIALIZED
                  81f166f0    00384000     TestAppEncoder.obj (.ccdData)

.bitsData 
*          0    8229a6f0    00020000     UNINITIALIZED
                  8229a6f0    00020000     TestAppEncoder.obj (.bitsData)

.ref_buffer 
*          0    822ba700    00020000     UNINITIALIZED
                  822ba700    00020000     TestAppEncoder.obj (.ref_buffer)


LINKER GENERATED COPY TABLES

__TI_cinit_table @ 0080e798 records: 28, size/record: 8, table size: 224
	.const.1: load addr=00809590, load size=00004231 bytes, run addr=00800000, run size=000047c8 bytes, compression=rle
	.fardata.1: load addr=0080d7c4, load size=0000088e bytes, run addr=00807090, run size=000016f8 bytes, compression=rle
	.const.4: load addr=0080e054, load size=000004be bytes, run addr=00804910, run size=000006a8 bytes, compression=rle
	.const.2: load addr=0080e514, load size=0000009d bytes, run addr=008047d0, run size=000000e8 bytes, compression=rle
	.const.5: load addr=0080e5b4, load size=00000059 bytes, run addr=00804fc0, run size=00000088 bytes, compression=rle
	.const.3: load addr=0080e610, load size=00000045 bytes, run addr=008048c0, run size=00000048 bytes, compression=rle
	.fardata.5: load addr=0080e658, load size=0000001a bytes, run addr=008087f0, run size=00000028 bytes, compression=rle
	.fardata.4: load addr=0080e674, load size=00000018 bytes, run addr=008087d0, run size=00000014 bytes, compression=rle
	.fardata.2: load addr=0080e68c, load size=00000016 bytes, run addr=00808790, run size=00000018 bytes, compression=rle
	.neardata: load addr=0080e6a4, load size=00000015 bytes, run addr=00809580, run size=00000010 bytes, compression=rle
	.fardata.3: load addr=0080e6bc, load size=0000000f bytes, run addr=008087b0, run size=00000014 bytes, compression=rle
	.const.6: load addr=0080e6cc, load size=0000000d bytes, run addr=00805050, run size=00000007 bytes, compression=rle
	.fardata.6: load addr=0080e6dc, load size=0000000d bytes, run addr=00808820, run size=00000008 bytes, compression=rle
	.fardata.7: load addr=0080e6ec, load size=0000000d bytes, run addr=00808830, run size=00000008 bytes, compression=rle
	.const.7: load addr=0080e6fc, load size=0000000c bytes, run addr=00805060, run size=00000006 bytes, compression=rle
	.const.9: load addr=0080e714, load size=0000000a bytes, run addr=00805080, run size=00000004 bytes, compression=rle
	.fardata.10: load addr=0080e720, load size=0000000a bytes, run addr=00808860, run size=00000004 bytes, compression=rle
	.fardata.12: load addr=0080e72c, load size=0000000a bytes, run addr=00808880, run size=00000004 bytes, compression=rle
	.const.8: load addr=0080e738, load size=00000009 bytes, run addr=00805070, run size=00000004 bytes, compression=rle
	.fardata.11: load addr=0080e744, load size=00000009 bytes, run addr=00808870, run size=00000004 bytes, compression=rle
	.fardata.8: load addr=0080e750, load size=00000009 bytes, run addr=00808840, run size=00000004 bytes, compression=rle
	.fardata.9: load addr=0080e75c, load size=00000009 bytes, run addr=00808850, run size=00000004 bytes, compression=rle
	.bitsData: load addr=0080e768, load size=00000008 bytes, run addr=8229a6f0, run size=00020000 bytes, compression=zero_init
	.bss: load addr=0080e770, load size=00000008 bytes, run addr=00809550, run size=00000030 bytes, compression=zero_init
	.ccdData: load addr=0080e778, load size=00000008 bytes, run addr=81f166f0, run size=00384000 bytes, compression=zero_init
	.far: load addr=0080e780, load size=00000008 bytes, run addr=80000000, run size=01f166e8 bytes, compression=zero_init
	.ref_buffer: load addr=0080e788, load size=00000008 bytes, run addr=822ba700, run size=00020000 bytes, compression=zero_init
	.taskStackSection: load addr=0080e790, load size=00000008 bytes, run addr=00808888, run size=00000800 bytes, compression=zero_init


LINKER GENERATED HANDLER TABLE

__TI_handler_table @ 0080e708 records: 3, size/record: 4, table size: 12
	index: 0, handler: __TI_zero_init
	index: 1, handler: __TI_decompress_rle24
	index: 2, handler: __TI_decompress_none


GLOBAL SYMBOLS: SORTED ALPHABETICALLY BY Name 

address    name
--------   ----
0c01ce60   ALG_create
0c01f8c0   ALG_delete
0c0239a0   C$$EXIT
0c022af8   C$$IO$$
0080957c   Capture_Height
00807fc0   DMJPGE_TIGEM_IDMJPGE
00809574   DRI_Interval
0c007da0   EncodeTask
00809558   EncodeTime
0c01efc0   GateMP_Params_init
0c01de60   GateMP_close
0c0211a0   GateMP_enter
0c021220   GateMP_leave
0c014c60   GateMP_openByAddr
0c011ae0   GateMP_sharedMemReq
0c020020   HOSTclose
0c01cd60   HOSTlseek
0c01df40   HOSTopen
0c01f080   HOSTread
0c0194e0   HOSTrename
0c01f140   HOSTunlink
0c01f200   HOSTwrite
0c01f2c0   HeapMemMP_Params_init
0c01b5e0   HeapMemMP_create
0c018520   HeapMemMP_sharedMemReq
00809584   ImageToEncode
81f1632c   InBuffers
0c016360   Initialize_original_buffer
81f164c0   InputBuffSize
0c0186e0   Ipc_start
0c00c200   NameServer_add
81f163f0   OutBuffers
0c0200c0   SharedRegion_getCacheLineSize
0c020160   SharedRegion_getHeap
0c020200   SharedRegion_getId
0c0202a0   SharedRegion_isCacheEnabled
0c023580   TSC_enable
0c023588   TSC_read
00808670   TSK_idle
0c020340   TestApp_CompareOutputData
0c021320   TestApp_EnableCache
0c01bfe0   TestApp_ReadInputData
0c0237a0   TestApp_SetDynamicParams
0c0237c0   TestApp_SetInitParams
0c01f380   TestApp_WriteOutputData
00809568   TotalBytes
0080956c   Total_BytesRead
0c00c860   _ALG_allocMemory
0c01f440   _ALG_freeMemory
0c0213a0   _Z11__TI_atexitPFYvPvES_S_
00800000   __ASM__
0080942c   __CIOBUF_
008000d0   __ISA__
008000f0   __PLAT__
00800120   __TARG__
0080e798   __TI_CINIT_Base
0080e878   __TI_CINIT_Limit
0080e708   __TI_Handler_Table_Base
0080e714   __TI_Handler_Table_Limit
00807088   __TI_STACK_END
00002000   __TI_STACK_SIZE
00809550   __TI_STATIC_BASE
00000001   __TI_args_main
0c0239e0   __TI_decompress_none
0c023a00   __TI_decompress_rle24
008086bc   __TI_enable_exit_profile_output
ffffffff   __TI_pprof_out_hndl
ffffffff   __TI_prof_data_size
ffffffff   __TI_prof_data_start
0c01e3a0   __TI_zero_init
00800150   __TRDR__
ffffffff   __binit__
0c00ce40   __c6xabi_divd
0c01e020   __c6xabi_divi
0c01c100   __c6xabi_divlli
0c01f5c0   __c6xabi_divu
0c019680   __c6xabi_divul
0c0165a0   __c6xabi_divull
0c021ea0   __c6xabi_frcmpyd_div
0c022d40   __c6xabi_isinf
0c021420   __c6xabi_llshl
0c021f00   __c6xabi_llshru
0c0237e0   __c6xabi_negll
0c0203e0   __c6xabi_remu
0c021f60   __c6xabi_remull
00809088   __c_args__
0c0213a0   __cxa_atexit
0c01f500   __cxa_finalize
0c023800   __cxa_ia64_exit
0c01e020   __divi
0c01f5c0   __divu
0c0203e0   __remu
0c023820   __xdc__init
00807b7c   __xdc__init__addr
0c022dc0   _args_main
00000200   _argsize
0c01ac40   _auto_init_elf
0c01b720   _buff_read
0c020480   _c_int00
0c01f680   _cleanup
008086b4   _cleanup_ptr
00804660   _ctypes_
0c01f740   _doflush
008086b8   _dtors_ptr
008085a8   _ft_end
00807b80   _ftable
00808078   _lock
0c023860   _nop
0c00f720   _printfi
0c01f800   _rd_ok
0c023900   _register_lock
0c023920   _register_unlock
0c00a2c0   _scanfi
00805088   _stack
0c021fc0   _subcull
81f164d0   _tmpnams
0080807c   _unlock
0c01c580   _wrt_ok
0c0239a0   abort
0c0239c0   atexit
0c01e1e0   atoi
ffffffff   binit
00809570   captureHeight
0c01e2c0   close
00809560   cycles
81f16258   dynamicParams
00808618   errno
0c01e480   exit
0c01c6a0   fclose
0c023a20   feof
0c01cf60   fflush
0c023a40   fgets
0c022020   fopen
0c021520   fprintf
0c01bae0   fputc
0c0134c0   fputs
0c015480   fread
0c022e80   free
0c01f980   fseek
0c0207a0   ftell
0c00f2a0   fwrite
81f16278   inArgs
81f166f0   inputData
81f14240   internalDataMemory
0080958c   internalDataMemorySize
0c022ec0   llabs
0c01fa40   lseek
0c01e640   ltoa
0c022f00   main
0c0215a0   malloc
0c01e720   memalign
0c022080   memccpy
0c0220e0   memcmp
0c020840   memcpy
0c01e800   memset
00809578   num_buf
0c01a4c0   open
81f1627c   outArgs
8229a6f0   outputData
00809588   pInternalDataMemory
81f16240   params
0c021620   printf
0c01bae0   putc
0c01fb00   read
0c0216a0   readmsg
0c022f40   readparamfile
822ba700   refData
0c021ba0   remove
008085b0   sTokenMap
0c01a640   setvbuf
0c0221a0   sscanf
81f1628c   status
0c022fc0   strcmp
0c023000   strlen
0c021720   strncpy
0c00df40   strtod
0c011740   strtol
0c00e460   strtold
0c00fb80   strtoll
0c0137c0   strtoul
0c010400   strtoull
00809550   t0
00809554   t1
0c00ffe0   ti_sdo_ipc_GateMP_Instance_finalize__F
0c008c40   ti_sdo_ipc_GateMP_Instance_init__F
00807090   ti_sdo_ipc_GateMP_Module_State_0_remoteCustom1Gates__A
00808840   ti_sdo_ipc_GateMP_Module_State_0_remoteCustom2Gates__A
00808230   ti_sdo_ipc_GateMP_Module_State_0_remoteSystemGates__A
00807890   ti_sdo_ipc_GateMP_Module__root__V
00807898   ti_sdo_ipc_GateMP_Module__state__V
00804c6c   ti_sdo_ipc_GateMP_Object__DESC__C
00804984   ti_sdo_ipc_GateMP_Object__PARAMS__C
0c01e8e0   ti_sdo_ipc_GateMP_Object__create__S
0c01e9c0   ti_sdo_ipc_GateMP_createLocal__F
0c017f60   ti_sdo_ipc_GateMP_getFreeResource__I
0c020980   ti_sdo_ipc_GateMP_getRegion0ReservedSize__F
0c0124e0   ti_sdo_ipc_GateMP_setRegion0Reserved__F
0c01ada0   ti_sdo_ipc_GateMP_start__F
008087b0   ti_sdo_ipc_Ipc_Module_State_0_procEntry__A
008078e0   ti_sdo_ipc_Ipc_Module__state__V
008078ec   ti_sdo_ipc_ListMP_Module__root__V
008078f4   ti_sdo_ipc_ListMP_Module__state__V
00808730   ti_sdo_ipc_MessageQ_Module_State_0_heaps__A
00808810   ti_sdo_ipc_MessageQ_Module_State_0_transports__A
008078f8   ti_sdo_ipc_MessageQ_Module__root__V
00807900   ti_sdo_ipc_MessageQ_Module__state__V
0c01fbc0   ti_sdo_ipc_MessageQ_Module_startup__E
0c01fbc0   ti_sdo_ipc_MessageQ_Module_startup__F
0080791c   ti_sdo_ipc_NameServerRemoteNotify_Module__root__V
0c018c20   ti_sdo_ipc_Notify_Instance_init__F
00808850   ti_sdo_ipc_Notify_Module_State_0_notifyHandles_0__A
00808860   ti_sdo_ipc_Notify_Module_State_0_notifyHandles__A
00807924   ti_sdo_ipc_Notify_Module__root__V
0080792c   ti_sdo_ipc_Notify_Module__state__V
0c0217a0   ti_sdo_ipc_Notify_Module_startup__E
0c0217a0   ti_sdo_ipc_Notify_Module_startup__F
00804c8c   ti_sdo_ipc_Notify_Object__DESC__C
00804f10   ti_sdo_ipc_Notify_Object__PARAMS__C
0c020a20   ti_sdo_ipc_Notify_Object__create__S
00808120   ti_sdo_ipc_SharedRegion_Module_State_0_regions__A
00807934   ti_sdo_ipc_SharedRegion_Module__state__V
0c019b60   ti_sdo_ipc_SharedRegion_reserveMemory__F
0c014980   ti_sdo_ipc_SharedRegion_start__F
0c023040   ti_sdo_ipc_gates_GateHWSem_Handle__label__S
008049e8   ti_sdo_ipc_gates_GateHWSem_Module__FXNS__C
00807938   ti_sdo_ipc_gates_GateHWSem_Module__root__V
0c01d060   ti_sdo_ipc_gates_GateHWSem_Module_startup__E
0c01d060   ti_sdo_ipc_gates_GateHWSem_Module_startup__F
00804cac   ti_sdo_ipc_gates_GateHWSem_Object__DESC__C
00804abc   ti_sdo_ipc_gates_GateHWSem_Object__PARAMS__C
0c01eaa0   ti_sdo_ipc_gates_GateHWSem_Object__create__S
0c022200   ti_sdo_ipc_gates_GateHWSem_Object__delete__S
0c01d160   ti_sdo_ipc_gates_GateHWSem_enter__E
0c01d160   ti_sdo_ipc_gates_GateHWSem_enter__F
0c023a60   ti_sdo_ipc_gates_GateHWSem_getReservedMask__E
0c023a60   ti_sdo_ipc_gates_GateHWSem_getReservedMask__F
0c023080   ti_sdo_ipc_gates_GateHWSem_leave__E
0c023080   ti_sdo_ipc_gates_GateHWSem_leave__F
0c023a80   ti_sdo_ipc_gates_GateHWSem_query__E
0c023a80   ti_sdo_ipc_gates_GateHWSem_query__F
00805070   ti_sdo_ipc_gates_GateHWSem_reservedMaskArr__A
00802288   ti_sdo_ipc_gates_GateHWSem_reservedMaskArr__C
0c023aa0   ti_sdo_ipc_gates_GateHWSem_sharedMemReq__E
0c023aa0   ti_sdo_ipc_gates_GateHWSem_sharedMemReq__F
0c0230c0   ti_sdo_ipc_gates_GateMPSupportNull_Handle__label__S
00804a14   ti_sdo_ipc_gates_GateMPSupportNull_Module__FXNS__C
00807940   ti_sdo_ipc_gates_GateMPSupportNull_Module__root__V
00804ccc   ti_sdo_ipc_gates_GateMPSupportNull_Object__DESC__C
00804ae0   ti_sdo_ipc_gates_GateMPSupportNull_Object__PARAMS__C
0c022260   ti_sdo_ipc_gates_GateMPSupportNull_Object__create__S
0c0222c0   ti_sdo_ipc_gates_GateMPSupportNull_Object__delete__S
0c023100   ti_sdo_ipc_gates_GateMPSupportNull_enter__E
0c023100   ti_sdo_ipc_gates_GateMPSupportNull_enter__F
0c023ac0   ti_sdo_ipc_gates_GateMPSupportNull_getReservedMask__E
0c023ac0   ti_sdo_ipc_gates_GateMPSupportNull_getReservedMask__F
0c023ae0   ti_sdo_ipc_gates_GateMPSupportNull_leave__E
0c023ae0   ti_sdo_ipc_gates_GateMPSupportNull_leave__F
0c023b00   ti_sdo_ipc_gates_GateMPSupportNull_query__E
0c023b00   ti_sdo_ipc_gates_GateMPSupportNull_query__F
0c023b20   ti_sdo_ipc_gates_GateMPSupportNull_sharedMemReq__E
0c023b20   ti_sdo_ipc_gates_GateMPSupportNull_sharedMemReq__F
0c023140   ti_sdo_ipc_gates_GatePeterson_Handle__label__S
0c022320   ti_sdo_ipc_gates_GatePeterson_Instance_finalize__F
0c010fe0   ti_sdo_ipc_gates_GatePeterson_Instance_init__F
00804a40   ti_sdo_ipc_gates_GatePeterson_Module__FXNS__C
00807948   ti_sdo_ipc_gates_GatePeterson_Module__root__V
00804cec   ti_sdo_ipc_gates_GatePeterson_Object__DESC__C
00804b04   ti_sdo_ipc_gates_GatePeterson_Object__PARAMS__C
0c01d260   ti_sdo_ipc_gates_GatePeterson_Object__create__S
0c022380   ti_sdo_ipc_gates_GatePeterson_Object__delete__S
0c01a940   ti_sdo_ipc_gates_GatePeterson_enter__E
0c01a940   ti_sdo_ipc_gates_GatePeterson_enter__F
0c023b40   ti_sdo_ipc_gates_GatePeterson_getReservedMask__E
0c023b40   ti_sdo_ipc_gates_GatePeterson_getReservedMask__F
0c020ac0   ti_sdo_ipc_gates_GatePeterson_leave__E
0c020ac0   ti_sdo_ipc_gates_GatePeterson_leave__F
0c023b60   ti_sdo_ipc_gates_GatePeterson_query__E
0c023b60   ti_sdo_ipc_gates_GatePeterson_query__F
0c0223e0   ti_sdo_ipc_gates_GatePeterson_sharedMemReq__E
0c0223e0   ti_sdo_ipc_gates_GatePeterson_sharedMemReq__F
0c023180   ti_sdo_ipc_heaps_HeapMemMP_Handle__label__S
0c01c7c0   ti_sdo_ipc_heaps_HeapMemMP_Instance_finalize__F
0c010c00   ti_sdo_ipc_heaps_HeapMemMP_Instance_init__F
00804a6c   ti_sdo_ipc_heaps_HeapMemMP_Module__FXNS__C
00807950   ti_sdo_ipc_heaps_HeapMemMP_Module__root__V
00807958   ti_sdo_ipc_heaps_HeapMemMP_Module__state__V
00804d0c   ti_sdo_ipc_heaps_HeapMemMP_Object__DESC__C
008049b8   ti_sdo_ipc_heaps_HeapMemMP_Object__PARAMS__C
0c01d360   ti_sdo_ipc_heaps_HeapMemMP_Object__create__S
0c022440   ti_sdo_ipc_heaps_HeapMemMP_Object__delete__S
0c010800   ti_sdo_ipc_heaps_HeapMemMP_alloc__E
0c010800   ti_sdo_ipc_heaps_HeapMemMP_alloc__F
0c012820   ti_sdo_ipc_heaps_HeapMemMP_free__E
0c012820   ti_sdo_ipc_heaps_HeapMemMP_free__F
0c01c8e0   ti_sdo_ipc_heaps_HeapMemMP_getStats__E
0c01c8e0   ti_sdo_ipc_heaps_HeapMemMP_getStats__F
0c023b80   ti_sdo_ipc_heaps_HeapMemMP_isBlocking__E
0c023b80   ti_sdo_ipc_heaps_HeapMemMP_isBlocking__F
0c0170c0   ti_sdo_ipc_heaps_HeapMemMP_postInit__I
0080228c   ti_sdo_ipc_interfaces_IGateMPSupport_Interface__BASE__C
00808870   ti_sdo_ipc_transports_TransportShmSetup_Module_State_0_handles__A
00807964   ti_sdo_ipc_transports_TransportShmSetup_Module__state__V
0080795c   ti_sdo_ipc_transports_TransportShm_Module__root__V
00807968   ti_sdo_utils_List_Module__root__V
00804d2c   ti_sdo_utils_List_Object__DESC__C
00804f28   ti_sdo_utils_List_Object__PARAMS__C
0c0224a0   ti_sdo_utils_List_Object__create__S
00807970   ti_sdo_utils_MultiProc_Module__state__V
80000000   ti_sdo_utils_NameServer_Module_State_0_nsRemoteHandle__A
00807974   ti_sdo_utils_NameServer_Module__root__V
0080797c   ti_sdo_utils_NameServer_Module__state__V
0c01d460   ti_sdo_utils_NameServer_Module_startup__E
0c01d460   ti_sdo_utils_NameServer_Module_startup__F
00807ee0   ti_sdo_utils_NameServer_Object__table__V
0c015c20   ti_sdo_utils_NameServer_removeLocal__I
00807984   ti_sysbios_BIOS_Module__state__V
0c020b60   ti_sysbios_BIOS_exitFunc__I
0c0172e0   ti_sysbios_BIOS_startFunc__I
0c023ba0   ti_sysbios_BIOS_start__E
0c022e00   ti_sysbios_family_c62_TaskSupport_buildTaskStack
0c023940   ti_sysbios_family_c62_TaskSupport_glue
0c0214a0   ti_sysbios_family_c62_TaskSupport_swap__E
008079a0   ti_sysbios_family_c64p_Exception_Module__state__V
0c022500   ti_sysbios_family_c64p_Exception_Module_startup__E
0c022500   ti_sysbios_family_c64p_Exception_Module_startup__F
0c01a7c0   ti_sysbios_family_c64p_Exception_dispatch__E
0c00b420   ti_sysbios_family_c64p_Exception_handler__I
0c017500   ti_sysbios_family_c64p_Exception_internalHandler__I
0c024000   ti_sysbios_family_c64p_Hwi0
0c024020   ti_sysbios_family_c64p_Hwi1
0c024140   ti_sysbios_family_c64p_Hwi10
0c024160   ti_sysbios_family_c64p_Hwi11
0c024180   ti_sysbios_family_c64p_Hwi12
0c0241a0   ti_sysbios_family_c64p_Hwi13
0c0241c0   ti_sysbios_family_c64p_Hwi14
0c0241e0   ti_sysbios_family_c64p_Hwi15
0c024040   ti_sysbios_family_c64p_Hwi2
0c024060   ti_sysbios_family_c64p_Hwi3
0c024080   ti_sysbios_family_c64p_Hwi4
0c0240a0   ti_sysbios_family_c64p_Hwi5
0c0240c0   ti_sysbios_family_c64p_Hwi6
0c0240e0   ti_sysbios_family_c64p_Hwi7
0c024100   ti_sysbios_family_c64p_Hwi8
0c024120   ti_sysbios_family_c64p_Hwi9
008079cc   ti_sysbios_family_c64p_Hwi_Module__root__V
008079d4   ti_sysbios_family_c64p_Hwi_Module__state__V
0c01bd60   ti_sysbios_family_c64p_Hwi_Module_startup__E
0c01bd60   ti_sysbios_family_c64p_Hwi_Module_startup__F
00808770   ti_sysbios_family_c64p_Hwi_Object__table__V
0c017d60   ti_sysbios_family_c64p_Hwi_dispatchAlways
0c01af00   ti_sysbios_family_c64p_Hwi_dispatchC__I
0c01bea0   ti_sysbios_family_c66_Cache_Module_startup__E
0c01bea0   ti_sysbios_family_c66_Cache_Module_startup__F
0c023bc0   ti_sysbios_family_c66_Cache_getMar__E
00805034   ti_sysbios_family_c66_Cache_initSize__C
00803f60   ti_sysbios_family_c66_Cache_marvalues__C
0c01fc80   ti_sysbios_family_c66_Cache_setMar__E
0c022560   ti_sysbios_family_c66_Cache_setSize__E
0c021820   ti_sysbios_family_c66_Cache_wbInvAll__E
0c023be0   ti_sysbios_family_c66_Cache_wbInv__E
0c022e40   ti_sysbios_family_xxx_Hwi_switchToIsrStack
0c023960   ti_sysbios_family_xxx_Hwi_switchToTaskStack
0c0231c0   ti_sysbios_gates_GateAll_Handle__label__S
00804b28   ti_sysbios_gates_GateAll_Module__FXNS__C
00807a34   ti_sysbios_gates_GateAll_Module__root__V
00804d4c   ti_sysbios_gates_GateAll_Object__DESC__C
00804f40   ti_sysbios_gates_GateAll_Object__PARAMS__C
0c0218a0   ti_sysbios_gates_GateAll_Object__create__S
0c0225c0   ti_sysbios_gates_GateAll_Object__delete__S
008087f0   ti_sysbios_gates_GateAll_Object__table__V
0c022620   ti_sysbios_gates_GateAll_enter__E
0c01d560   ti_sysbios_gates_GateAll_leave__E
0c023c00   ti_sysbios_gates_GateAll_query__E
0c023c00   ti_sysbios_gates_GateAll_query__F
00807a3c   ti_sysbios_gates_GateHwi_Module__root__V
0c023200   ti_sysbios_gates_GateMutexPri_Handle__label__S
0c023240   ti_sysbios_gates_GateMutexPri_Instance_finalize__F
00804b4c   ti_sysbios_gates_GateMutexPri_Module__FXNS__C
00807a4c   ti_sysbios_gates_GateMutexPri_Module__root__V
00804d6c   ti_sysbios_gates_GateMutexPri_Object__DESC__C
00804f58   ti_sysbios_gates_GateMutexPri_Object__PARAMS__C
0c020c00   ti_sysbios_gates_GateMutexPri_Object__create__S
0c022680   ti_sysbios_gates_GateMutexPri_Object__delete__S
00808790   ti_sysbios_gates_GateMutexPri_Object__table__V
0c011e40   ti_sysbios_gates_GateMutexPri_enter__E
0c018de0   ti_sysbios_gates_GateMutexPri_leave__E
0c023c20   ti_sysbios_gates_GateMutexPri_query__E
0c023c20   ti_sysbios_gates_GateMutexPri_query__F
0c023280   ti_sysbios_gates_GateMutex_Handle__label__S
0c0232c0   ti_sysbios_gates_GateMutex_Instance_finalize__F
00804b70   ti_sysbios_gates_GateMutex_Module__FXNS__C
00807a44   ti_sysbios_gates_GateMutex_Module__root__V
00804d8c   ti_sysbios_gates_GateMutex_Object__DESC__C
00804f70   ti_sysbios_gates_GateMutex_Object__PARAMS__C
0c020ca0   ti_sysbios_gates_GateMutex_Object__create__S
0c0226e0   ti_sysbios_gates_GateMutex_Object__delete__S
008086c0   ti_sysbios_gates_GateMutex_Object__table__V
0c01eb80   ti_sysbios_gates_GateMutex_enter__E
0c023c40   ti_sysbios_gates_GateMutex_leave__E
0c023c60   ti_sysbios_gates_GateMutex_query__E
0c023c60   ti_sysbios_gates_GateMutex_query__F
0c023300   ti_sysbios_gates_GateSwi_Handle__label__S
00804b94   ti_sysbios_gates_GateSwi_Module__FXNS__C
00807a54   ti_sysbios_gates_GateSwi_Module__root__V
00804dac   ti_sysbios_gates_GateSwi_Object__DESC__C
00804f88   ti_sysbios_gates_GateSwi_Object__PARAMS__C
0c022740   ti_sysbios_gates_GateSwi_Object__create__S
0c0227a0   ti_sysbios_gates_GateSwi_Object__delete__S
00808800   ti_sysbios_gates_GateSwi_Object__table__V
0c020d40   ti_sysbios_gates_GateSwi_enter__E
0c01ec60   ti_sysbios_gates_GateSwi_leave__E
0c023c80   ti_sysbios_gates_GateSwi_query__E
0c023c80   ti_sysbios_gates_GateSwi_query__F
00807a5c   ti_sysbios_hal_Hwi_Module__root__V
0c023340   ti_sysbios_hal_Hwi_Module_startup__E
0c023340   ti_sysbios_hal_Hwi_Module_startup__F
00808820   ti_sysbios_hal_Hwi_Object__table__V
0c021920   ti_sysbios_hal_Hwi_checkStack
0c022800   ti_sysbios_hal_Hwi_initStack
00807a64   ti_sysbios_hal_Timer_Module__root__V
0c023380   ti_sysbios_hal_Timer_Module_startup__E
0c023380   ti_sysbios_hal_Timer_Module_startup__F
00808830   ti_sysbios_hal_Timer_Object__table__V
0c0233c0   ti_sysbios_heaps_HeapMem_Handle__label__S
80000008   ti_sysbios_heaps_HeapMem_Instance_State_0_buf__A
00804a94   ti_sysbios_heaps_HeapMem_Module__FXNS__C
00807a6c   ti_sysbios_heaps_HeapMem_Module__root__V
00804dcc   ti_sysbios_heaps_HeapMem_Object__DESC__C
00804dec   ti_sysbios_heaps_HeapMem_Object__PARAMS__C
0c01d660   ti_sysbios_heaps_HeapMem_Object__create__S
0c022860   ti_sysbios_heaps_HeapMem_Object__delete__S
008087d0   ti_sysbios_heaps_HeapMem_Object__table__V
0c018160   ti_sysbios_heaps_HeapMem_alloc__E
0c015ea0   ti_sysbios_heaps_HeapMem_free__E
0c01fd40   ti_sysbios_heaps_HeapMem_getStats__E
0c023400   ti_sysbios_heaps_HeapMem_init__I
0c023ca0   ti_sysbios_heaps_HeapMem_isBlocking__E
0c020de0   ti_sysbios_knl_Clock_Instance_finalize__F
00807a74   ti_sysbios_knl_Clock_Module__root__V
00807a7c   ti_sysbios_knl_Clock_Module__state__V
0c023440   ti_sysbios_knl_Clock_Module_startup__E
0c023440   ti_sysbios_knl_Clock_Module_startup__F
00804e0c   ti_sysbios_knl_Clock_Object__DESC__C
00804bb8   ti_sysbios_knl_Clock_Object__PARAMS__C
0c01b060   ti_sysbios_knl_Clock_Object__create__S
0c0228c0   ti_sysbios_knl_Clock_doTick__I
0c01ca00   ti_sysbios_knl_Clock_workFunc__E
00805080   ti_sysbios_knl_Idle_funcList__A
0c0219a0   ti_sysbios_knl_Idle_loop__E
00807a98   ti_sysbios_knl_Queue_Module__root__V
00804e2c   ti_sysbios_knl_Queue_Object__DESC__C
00804fa0   ti_sysbios_knl_Queue_Object__PARAMS__C
0c022920   ti_sysbios_knl_Queue_Object__create__S
0c023480   ti_sysbios_knl_Semaphore_Instance_finalize__F
00807aa0   ti_sysbios_knl_Semaphore_Module__root__V
00804e4c   ti_sysbios_knl_Semaphore_Object__DESC__C
00804bdc   ti_sysbios_knl_Semaphore_Object__PARAMS__C
0c01ed40   ti_sysbios_knl_Semaphore_Object__create__S
0c021a20   ti_sysbios_knl_Semaphore_pendTimeout__I
0c012b60   ti_sysbios_knl_Semaphore_pend__E
0c01d760   ti_sysbios_knl_Semaphore_post__E
008082b0   ti_sysbios_knl_Swi_Module_State_0_readyQ__A
00807aa8   ti_sysbios_knl_Swi_Module__root__V
00807ab0   ti_sysbios_knl_Swi_Module__state__V
0c023cc0   ti_sysbios_knl_Swi_Module_startup__E
0c023cc0   ti_sysbios_knl_Swi_Module_startup__F
00808700   ti_sysbios_knl_Swi_Object__table__V
0c021aa0   ti_sysbios_knl_Swi_post__E
0c01d860   ti_sysbios_knl_Swi_restoreHwi__E
0c01fe00   ti_sysbios_knl_Swi_run__I
0c018340   ti_sysbios_knl_Swi_schedule__I
81f0f010   ti_sysbios_knl_Task_Instance_State_0_hookEnv__A
00808888   ti_sysbios_knl_Task_Instance_State_0_stack__A
0c013ac0   ti_sysbios_knl_Task_Instance_finalize__F
0c016c60   ti_sysbios_knl_Task_Instance_init__F
00808330   ti_sysbios_knl_Task_Module_State_0_readyQ__A
00807acc   ti_sysbios_knl_Task_Module__root__V
00807ad4   ti_sysbios_knl_Task_Module__state__V
0c022980   ti_sysbios_knl_Task_Module_startup__E
0c022980   ti_sysbios_knl_Task_Module_startup__F
00804e6c   ti_sysbios_knl_Task_Object__DESC__C
0080494c   ti_sysbios_knl_Task_Object__PARAMS__C
0c01d960   ti_sysbios_knl_Task_Object__create__S
00808670   ti_sysbios_knl_Task_Object__table__V
0c020e80   ti_sysbios_knl_Task_Params__init__S
0c0229e0   ti_sysbios_knl_Task_allBlockedFunction__I
0c018fa0   ti_sysbios_knl_Task_checkStacks__E
0c022a40   ti_sysbios_knl_Task_enter__I
0c01b1c0   ti_sysbios_knl_Task_exit__E
00804fc0   ti_sysbios_knl_Task_hooks__A
0c017720   ti_sysbios_knl_Task_postInit__I
0c01cb20   ti_sysbios_knl_Task_schedule__I
0c016100   ti_sysbios_knl_Task_setPri__E
0c01da60   ti_sysbios_knl_Task_startup__E
0c021b20   ti_sysbios_knl_Task_unblockI__E
00807b08   ti_sysbios_syncs_SyncSem_Module__root__V
00807d60   ti_sysbios_timers_timer64_Timer_Module_State_0_device__A
008083b0   ti_sysbios_timers_timer64_Timer_Module_State_0_gctrl__A
00808430   ti_sysbios_timers_timer64_Timer_Module_State_0_handles__A
008084b0   ti_sysbios_timers_timer64_Timer_Module_State_0_intFreqs__A
00807b10   ti_sysbios_timers_timer64_Timer_Module__root__V
00807b18   ti_sysbios_timers_timer64_Timer_Module__state__V
0c013dc0   ti_sysbios_timers_timer64_Timer_Module_startup__E
0c013dc0   ti_sysbios_timers_timer64_Timer_Module_startup__F
00808620   ti_sysbios_timers_timer64_Timer_Object__table__V
0c019160   ti_sysbios_timers_timer64_Timer_setPeriodMicroSecs__E
0c019d00   ti_sysbios_timers_timer64_Timer_start__E
0c01ee20   ti_sysbios_timers_timer64_Timer_stop__E
0c023540   ti_sysbios_xdcruntime_GateThreadSupport_Instance_finalize__F
00807b2c   ti_sysbios_xdcruntime_GateThreadSupport_Module__root__V
00804e8c   ti_sysbios_xdcruntime_GateThreadSupport_Object__DESC__C
00804fd8   ti_sysbios_xdcruntime_GateThreadSupport_Object__PARAMS__C
0c020f20   ti_sysbios_xdcruntime_GateThreadSupport_Object__create__S
0c023c20   ti_sysbios_xdcruntime_GateThreadSupport_query__E
0c023c20   ti_sysbios_xdcruntime_GateThreadSupport_query__F
00809580   total_size
0c021ba0   unlink
0c01fec0   write
0c022aa0   writemsg
0c021c20   xdc_runtime_Assert_raise__I
0c017940   xdc_runtime_Core_createObject__I
0c01b320   xdc_runtime_Core_deleteObject__I
00807b34   xdc_runtime_Error_Module__state__V
0c020fc0   xdc_runtime_Error_print__E
0c020fc0   xdc_runtime_Error_print__F
0c01aac0   xdc_runtime_Error_raiseX__E
0c01aac0   xdc_runtime_Error_raiseX__F
0c0235c0   xdc_runtime_GateNull_Handle__label__S
00804c00   xdc_runtime_GateNull_Module__FXNS__C
00807b38   xdc_runtime_GateNull_Module__root__V
00804eac   xdc_runtime_GateNull_Object__DESC__C
00804ff0   xdc_runtime_GateNull_Object__PARAMS__C
0c022b00   xdc_runtime_GateNull_Object__create__S
0c022b60   xdc_runtime_GateNull_Object__delete__S
00808880   xdc_runtime_GateNull_Object__table__V
0c023ce0   xdc_runtime_GateNull_enter__E
0c023ce0   xdc_runtime_GateNull_enter__F
0c023d00   xdc_runtime_GateNull_leave__E
0c023d00   xdc_runtime_GateNull_leave__F
0c023d20   xdc_runtime_GateNull_query__E
0c023d20   xdc_runtime_GateNull_query__F
00804508   xdc_runtime_IGateProvider_Interface__BASE__C
0080450c   xdc_runtime_IHeap_Interface__BASE__C
0080465c   xdc_runtime_IModule_Interface__BASE__C
00807b40   xdc_runtime_Memory_Module__state__V
0c01db60   xdc_runtime_Memory_alloc__F
0c022bc0   xdc_runtime_Memory_calloc__E
0c022bc0   xdc_runtime_Memory_calloc__F
0c023600   xdc_runtime_Memory_free__E
0c023600   xdc_runtime_Memory_free__F
00807b44   xdc_runtime_Registry_Module__state__V
00807b4c   xdc_runtime_Startup_Module__state__V
00000001   xdc_runtime_Startup__EXECFXN__C
00000001   xdc_runtime_Startup__RESETFXN__C
0c021ca0   xdc_runtime_Startup_exec__E
0c021ca0   xdc_runtime_Startup_exec__F
0c023d60   xdc_runtime_Startup_exec__I
00805040   xdc_runtime_Startup_firstFxns__A
0c023d80   xdc_runtime_Startup_reset__I
00804ef0   xdc_runtime_Startup_sfxnRts__A
00804910   xdc_runtime_Startup_sfxnTab__A
0c019320   xdc_runtime_Startup_startMods__I
81f0f020   xdc_runtime_SysMin_Module_State_0_outbuf__A
00807b54   xdc_runtime_SysMin_Module__state__V
0c023640   xdc_runtime_SysMin_Module_startup__E
0c023640   xdc_runtime_SysMin_Module_startup__F
0c01cc40   xdc_runtime_SysMin_flush__E
0c01cc40   xdc_runtime_SysMin_flush__F
0c022c20   xdc_runtime_SysMin_putch__E
0c022c20   xdc_runtime_SysMin_putch__F
00808750   xdc_runtime_System_Module_State_0_atexitHandlers__A
00807b60   xdc_runtime_System_Module__state__V
0c023da0   xdc_runtime_System_Module_startup__E
0c023da0   xdc_runtime_System_Module_startup__F
0c01cc40   xdc_runtime_System_SupportProxy_flush__E
0c021060   xdc_runtime_System_abort__E
0c021060   xdc_runtime_System_abort__F
0c023680   xdc_runtime_System_aprintf__E
0c022c80   xdc_runtime_System_atexit__E
0c022c80   xdc_runtime_System_atexit__F
0c009840   xdc_runtime_System_doPrint__I
0c023dc0   xdc_runtime_System_exit__E
0c023dc0   xdc_runtime_System_exit__F
0c01cc40   xdc_runtime_System_flush__E
0c01cc40   xdc_runtime_System_flush__F
0c0140c0   xdc_runtime_System_printfExtend__I
0c0236c0   xdc_runtime_System_printf__E
0c021d20   xdc_runtime_System_rtsExit__I
00807b6c   xdc_runtime_Text_Module__state__V
00800000   xdc_runtime_Text_charTab__A
00804510   xdc_runtime_Text_nodeTab__A
0c021da0   xdc_runtime_Text_printVisFxn__I
0c01dc60   xdc_runtime_Text_putMod__F
0c019ea0   xdc_runtime_Text_putSite__E
0c019ea0   xdc_runtime_Text_putSite__F
0c01b480   xdc_runtime_Text_visitRope2__I
0c023de0   xdc_runtime_Text_visitRope__I
0c021100   xdc_runtime_Text_xprintf__I
0c023700   xdc_runtime_knl_GateThread_Handle__label__S
0c021e20   xdc_runtime_knl_GateThread_Instance_finalize__F
00804c24   xdc_runtime_knl_GateThread_Module__FXNS__C
00807b74   xdc_runtime_knl_GateThread_Module__root__V
00804ecc   xdc_runtime_knl_GateThread_Object__DESC__C
00805008   xdc_runtime_knl_GateThread_Object__PARAMS__C
0c01dd60   xdc_runtime_knl_GateThread_Object__create__S
0c022ce0   xdc_runtime_knl_GateThread_Object__delete__S
0c023c20   xdc_runtime_knl_GateThread_Proxy_query__E
0c023e00   xdc_runtime_knl_GateThread_enter__E
0c023e00   xdc_runtime_knl_GateThread_enter__F
0c023e20   xdc_runtime_knl_GateThread_leave__E
0c023e20   xdc_runtime_knl_GateThread_leave__F
0c023c20   xdc_runtime_knl_GateThread_query__E
0c023c20   xdc_runtime_knl_GateThread_query__F


GLOBAL SYMBOLS: SORTED BY Symbol Address 

address    name
--------   ----
00000001   __TI_args_main
00000001   xdc_runtime_Startup__EXECFXN__C
00000001   xdc_runtime_Startup__RESETFXN__C
00000200   _argsize
00002000   __TI_STACK_SIZE
00800000   __ASM__
00800000   xdc_runtime_Text_charTab__A
008000d0   __ISA__
008000f0   __PLAT__
00800120   __TARG__
00800150   __TRDR__
00802288   ti_sdo_ipc_gates_GateHWSem_reservedMaskArr__C
0080228c   ti_sdo_ipc_interfaces_IGateMPSupport_Interface__BASE__C
00803f60   ti_sysbios_family_c66_Cache_marvalues__C
00804508   xdc_runtime_IGateProvider_Interface__BASE__C
0080450c   xdc_runtime_IHeap_Interface__BASE__C
00804510   xdc_runtime_Text_nodeTab__A
0080465c   xdc_runtime_IModule_Interface__BASE__C
00804660   _ctypes_
00804910   xdc_runtime_Startup_sfxnTab__A
0080494c   ti_sysbios_knl_Task_Object__PARAMS__C
00804984   ti_sdo_ipc_GateMP_Object__PARAMS__C
008049b8   ti_sdo_ipc_heaps_HeapMemMP_Object__PARAMS__C
008049e8   ti_sdo_ipc_gates_GateHWSem_Module__FXNS__C
00804a14   ti_sdo_ipc_gates_GateMPSupportNull_Module__FXNS__C
00804a40   ti_sdo_ipc_gates_GatePeterson_Module__FXNS__C
00804a6c   ti_sdo_ipc_heaps_HeapMemMP_Module__FXNS__C
00804a94   ti_sysbios_heaps_HeapMem_Module__FXNS__C
00804abc   ti_sdo_ipc_gates_GateHWSem_Object__PARAMS__C
00804ae0   ti_sdo_ipc_gates_GateMPSupportNull_Object__PARAMS__C
00804b04   ti_sdo_ipc_gates_GatePeterson_Object__PARAMS__C
00804b28   ti_sysbios_gates_GateAll_Module__FXNS__C
00804b4c   ti_sysbios_gates_GateMutexPri_Module__FXNS__C
00804b70   ti_sysbios_gates_GateMutex_Module__FXNS__C
00804b94   ti_sysbios_gates_GateSwi_Module__FXNS__C
00804bb8   ti_sysbios_knl_Clock_Object__PARAMS__C
00804bdc   ti_sysbios_knl_Semaphore_Object__PARAMS__C
00804c00   xdc_runtime_GateNull_Module__FXNS__C
00804c24   xdc_runtime_knl_GateThread_Module__FXNS__C
00804c6c   ti_sdo_ipc_GateMP_Object__DESC__C
00804c8c   ti_sdo_ipc_Notify_Object__DESC__C
00804cac   ti_sdo_ipc_gates_GateHWSem_Object__DESC__C
00804ccc   ti_sdo_ipc_gates_GateMPSupportNull_Object__DESC__C
00804cec   ti_sdo_ipc_gates_GatePeterson_Object__DESC__C
00804d0c   ti_sdo_ipc_heaps_HeapMemMP_Object__DESC__C
00804d2c   ti_sdo_utils_List_Object__DESC__C
00804d4c   ti_sysbios_gates_GateAll_Object__DESC__C
00804d6c   ti_sysbios_gates_GateMutexPri_Object__DESC__C
00804d8c   ti_sysbios_gates_GateMutex_Object__DESC__C
00804dac   ti_sysbios_gates_GateSwi_Object__DESC__C
00804dcc   ti_sysbios_heaps_HeapMem_Object__DESC__C
00804dec   ti_sysbios_heaps_HeapMem_Object__PARAMS__C
00804e0c   ti_sysbios_knl_Clock_Object__DESC__C
00804e2c   ti_sysbios_knl_Queue_Object__DESC__C
00804e4c   ti_sysbios_knl_Semaphore_Object__DESC__C
00804e6c   ti_sysbios_knl_Task_Object__DESC__C
00804e8c   ti_sysbios_xdcruntime_GateThreadSupport_Object__DESC__C
00804eac   xdc_runtime_GateNull_Object__DESC__C
00804ecc   xdc_runtime_knl_GateThread_Object__DESC__C
00804ef0   xdc_runtime_Startup_sfxnRts__A
00804f10   ti_sdo_ipc_Notify_Object__PARAMS__C
00804f28   ti_sdo_utils_List_Object__PARAMS__C
00804f40   ti_sysbios_gates_GateAll_Object__PARAMS__C
00804f58   ti_sysbios_gates_GateMutexPri_Object__PARAMS__C
00804f70   ti_sysbios_gates_GateMutex_Object__PARAMS__C
00804f88   ti_sysbios_gates_GateSwi_Object__PARAMS__C
00804fa0   ti_sysbios_knl_Queue_Object__PARAMS__C
00804fc0   ti_sysbios_knl_Task_hooks__A
00804fd8   ti_sysbios_xdcruntime_GateThreadSupport_Object__PARAMS__C
00804ff0   xdc_runtime_GateNull_Object__PARAMS__C
00805008   xdc_runtime_knl_GateThread_Object__PARAMS__C
00805034   ti_sysbios_family_c66_Cache_initSize__C
00805040   xdc_runtime_Startup_firstFxns__A
00805070   ti_sdo_ipc_gates_GateHWSem_reservedMaskArr__A
00805080   ti_sysbios_knl_Idle_funcList__A
00805088   _stack
00807088   __TI_STACK_END
00807090   ti_sdo_ipc_GateMP_Module_State_0_remoteCustom1Gates__A
00807890   ti_sdo_ipc_GateMP_Module__root__V
00807898   ti_sdo_ipc_GateMP_Module__state__V
008078e0   ti_sdo_ipc_Ipc_Module__state__V
008078ec   ti_sdo_ipc_ListMP_Module__root__V
008078f4   ti_sdo_ipc_ListMP_Module__state__V
008078f8   ti_sdo_ipc_MessageQ_Module__root__V
00807900   ti_sdo_ipc_MessageQ_Module__state__V
0080791c   ti_sdo_ipc_NameServerRemoteNotify_Module__root__V
00807924   ti_sdo_ipc_Notify_Module__root__V
0080792c   ti_sdo_ipc_Notify_Module__state__V
00807934   ti_sdo_ipc_SharedRegion_Module__state__V
00807938   ti_sdo_ipc_gates_GateHWSem_Module__root__V
00807940   ti_sdo_ipc_gates_GateMPSupportNull_Module__root__V
00807948   ti_sdo_ipc_gates_GatePeterson_Module__root__V
00807950   ti_sdo_ipc_heaps_HeapMemMP_Module__root__V
00807958   ti_sdo_ipc_heaps_HeapMemMP_Module__state__V
0080795c   ti_sdo_ipc_transports_TransportShm_Module__root__V
00807964   ti_sdo_ipc_transports_TransportShmSetup_Module__state__V
00807968   ti_sdo_utils_List_Module__root__V
00807970   ti_sdo_utils_MultiProc_Module__state__V
00807974   ti_sdo_utils_NameServer_Module__root__V
0080797c   ti_sdo_utils_NameServer_Module__state__V
00807984   ti_sysbios_BIOS_Module__state__V
008079a0   ti_sysbios_family_c64p_Exception_Module__state__V
008079cc   ti_sysbios_family_c64p_Hwi_Module__root__V
008079d4   ti_sysbios_family_c64p_Hwi_Module__state__V
00807a34   ti_sysbios_gates_GateAll_Module__root__V
00807a3c   ti_sysbios_gates_GateHwi_Module__root__V
00807a44   ti_sysbios_gates_GateMutex_Module__root__V
00807a4c   ti_sysbios_gates_GateMutexPri_Module__root__V
00807a54   ti_sysbios_gates_GateSwi_Module__root__V
00807a5c   ti_sysbios_hal_Hwi_Module__root__V
00807a64   ti_sysbios_hal_Timer_Module__root__V
00807a6c   ti_sysbios_heaps_HeapMem_Module__root__V
00807a74   ti_sysbios_knl_Clock_Module__root__V
00807a7c   ti_sysbios_knl_Clock_Module__state__V
00807a98   ti_sysbios_knl_Queue_Module__root__V
00807aa0   ti_sysbios_knl_Semaphore_Module__root__V
00807aa8   ti_sysbios_knl_Swi_Module__root__V
00807ab0   ti_sysbios_knl_Swi_Module__state__V
00807acc   ti_sysbios_knl_Task_Module__root__V
00807ad4   ti_sysbios_knl_Task_Module__state__V
00807b08   ti_sysbios_syncs_SyncSem_Module__root__V
00807b10   ti_sysbios_timers_timer64_Timer_Module__root__V
00807b18   ti_sysbios_timers_timer64_Timer_Module__state__V
00807b2c   ti_sysbios_xdcruntime_GateThreadSupport_Module__root__V
00807b34   xdc_runtime_Error_Module__state__V
00807b38   xdc_runtime_GateNull_Module__root__V
00807b40   xdc_runtime_Memory_Module__state__V
00807b44   xdc_runtime_Registry_Module__state__V
00807b4c   xdc_runtime_Startup_Module__state__V
00807b54   xdc_runtime_SysMin_Module__state__V
00807b60   xdc_runtime_System_Module__state__V
00807b6c   xdc_runtime_Text_Module__state__V
00807b74   xdc_runtime_knl_GateThread_Module__root__V
00807b7c   __xdc__init__addr
00807b80   _ftable
00807d60   ti_sysbios_timers_timer64_Timer_Module_State_0_device__A
00807ee0   ti_sdo_utils_NameServer_Object__table__V
00807fc0   DMJPGE_TIGEM_IDMJPGE
00808078   _lock
0080807c   _unlock
00808120   ti_sdo_ipc_SharedRegion_Module_State_0_regions__A
00808230   ti_sdo_ipc_GateMP_Module_State_0_remoteSystemGates__A
008082b0   ti_sysbios_knl_Swi_Module_State_0_readyQ__A
00808330   ti_sysbios_knl_Task_Module_State_0_readyQ__A
008083b0   ti_sysbios_timers_timer64_Timer_Module_State_0_gctrl__A
00808430   ti_sysbios_timers_timer64_Timer_Module_State_0_handles__A
008084b0   ti_sysbios_timers_timer64_Timer_Module_State_0_intFreqs__A
008085a8   _ft_end
008085b0   sTokenMap
00808618   errno
00808620   ti_sysbios_timers_timer64_Timer_Object__table__V
00808670   TSK_idle
00808670   ti_sysbios_knl_Task_Object__table__V
008086b4   _cleanup_ptr
008086b8   _dtors_ptr
008086bc   __TI_enable_exit_profile_output
008086c0   ti_sysbios_gates_GateMutex_Object__table__V
00808700   ti_sysbios_knl_Swi_Object__table__V
00808730   ti_sdo_ipc_MessageQ_Module_State_0_heaps__A
00808750   xdc_runtime_System_Module_State_0_atexitHandlers__A
00808770   ti_sysbios_family_c64p_Hwi_Object__table__V
00808790   ti_sysbios_gates_GateMutexPri_Object__table__V
008087b0   ti_sdo_ipc_Ipc_Module_State_0_procEntry__A
008087d0   ti_sysbios_heaps_HeapMem_Object__table__V
008087f0   ti_sysbios_gates_GateAll_Object__table__V
00808800   ti_sysbios_gates_GateSwi_Object__table__V
00808810   ti_sdo_ipc_MessageQ_Module_State_0_transports__A
00808820   ti_sysbios_hal_Hwi_Object__table__V
00808830   ti_sysbios_hal_Timer_Object__table__V
00808840   ti_sdo_ipc_GateMP_Module_State_0_remoteCustom2Gates__A
00808850   ti_sdo_ipc_Notify_Module_State_0_notifyHandles_0__A
00808860   ti_sdo_ipc_Notify_Module_State_0_notifyHandles__A
00808870   ti_sdo_ipc_transports_TransportShmSetup_Module_State_0_handles__A
00808880   xdc_runtime_GateNull_Object__table__V
00808888   ti_sysbios_knl_Task_Instance_State_0_stack__A
00809088   __c_args__
0080942c   __CIOBUF_
00809550   __TI_STATIC_BASE
00809550   t0
00809554   t1
00809558   EncodeTime
00809560   cycles
00809568   TotalBytes
0080956c   Total_BytesRead
00809570   captureHeight
00809574   DRI_Interval
00809578   num_buf
0080957c   Capture_Height
00809580   total_size
00809584   ImageToEncode
00809588   pInternalDataMemory
0080958c   internalDataMemorySize
0080e708   __TI_Handler_Table_Base
0080e714   __TI_Handler_Table_Limit
0080e798   __TI_CINIT_Base
0080e878   __TI_CINIT_Limit
0c007da0   EncodeTask
0c008c40   ti_sdo_ipc_GateMP_Instance_init__F
0c009840   xdc_runtime_System_doPrint__I
0c00a2c0   _scanfi
0c00b420   ti_sysbios_family_c64p_Exception_handler__I
0c00c200   NameServer_add
0c00c860   _ALG_allocMemory
0c00ce40   __c6xabi_divd
0c00df40   strtod
0c00e460   strtold
0c00f2a0   fwrite
0c00f720   _printfi
0c00fb80   strtoll
0c00ffe0   ti_sdo_ipc_GateMP_Instance_finalize__F
0c010400   strtoull
0c010800   ti_sdo_ipc_heaps_HeapMemMP_alloc__E
0c010800   ti_sdo_ipc_heaps_HeapMemMP_alloc__F
0c010c00   ti_sdo_ipc_heaps_HeapMemMP_Instance_init__F
0c010fe0   ti_sdo_ipc_gates_GatePeterson_Instance_init__F
0c011740   strtol
0c011ae0   GateMP_sharedMemReq
0c011e40   ti_sysbios_gates_GateMutexPri_enter__E
0c0124e0   ti_sdo_ipc_GateMP_setRegion0Reserved__F
0c012820   ti_sdo_ipc_heaps_HeapMemMP_free__E
0c012820   ti_sdo_ipc_heaps_HeapMemMP_free__F
0c012b60   ti_sysbios_knl_Semaphore_pend__E
0c0134c0   fputs
0c0137c0   strtoul
0c013ac0   ti_sysbios_knl_Task_Instance_finalize__F
0c013dc0   ti_sysbios_timers_timer64_Timer_Module_startup__E
0c013dc0   ti_sysbios_timers_timer64_Timer_Module_startup__F
0c0140c0   xdc_runtime_System_printfExtend__I
0c014980   ti_sdo_ipc_SharedRegion_start__F
0c014c60   GateMP_openByAddr
0c015480   fread
0c015c20   ti_sdo_utils_NameServer_removeLocal__I
0c015ea0   ti_sysbios_heaps_HeapMem_free__E
0c016100   ti_sysbios_knl_Task_setPri__E
0c016360   Initialize_original_buffer
0c0165a0   __c6xabi_divull
0c016c60   ti_sysbios_knl_Task_Instance_init__F
0c0170c0   ti_sdo_ipc_heaps_HeapMemMP_postInit__I
0c0172e0   ti_sysbios_BIOS_startFunc__I
0c017500   ti_sysbios_family_c64p_Exception_internalHandler__I
0c017720   ti_sysbios_knl_Task_postInit__I
0c017940   xdc_runtime_Core_createObject__I
0c017d60   ti_sysbios_family_c64p_Hwi_dispatchAlways
0c017f60   ti_sdo_ipc_GateMP_getFreeResource__I
0c018160   ti_sysbios_heaps_HeapMem_alloc__E
0c018340   ti_sysbios_knl_Swi_schedule__I
0c018520   HeapMemMP_sharedMemReq
0c0186e0   Ipc_start
0c018c20   ti_sdo_ipc_Notify_Instance_init__F
0c018de0   ti_sysbios_gates_GateMutexPri_leave__E
0c018fa0   ti_sysbios_knl_Task_checkStacks__E
0c019160   ti_sysbios_timers_timer64_Timer_setPeriodMicroSecs__E
0c019320   xdc_runtime_Startup_startMods__I
0c0194e0   HOSTrename
0c019680   __c6xabi_divul
0c019b60   ti_sdo_ipc_SharedRegion_reserveMemory__F
0c019d00   ti_sysbios_timers_timer64_Timer_start__E
0c019ea0   xdc_runtime_Text_putSite__E
0c019ea0   xdc_runtime_Text_putSite__F
0c01a4c0   open
0c01a640   setvbuf
0c01a7c0   ti_sysbios_family_c64p_Exception_dispatch__E
0c01a940   ti_sdo_ipc_gates_GatePeterson_enter__E
0c01a940   ti_sdo_ipc_gates_GatePeterson_enter__F
0c01aac0   xdc_runtime_Error_raiseX__E
0c01aac0   xdc_runtime_Error_raiseX__F
0c01ac40   _auto_init_elf
0c01ada0   ti_sdo_ipc_GateMP_start__F
0c01af00   ti_sysbios_family_c64p_Hwi_dispatchC__I
0c01b060   ti_sysbios_knl_Clock_Object__create__S
0c01b1c0   ti_sysbios_knl_Task_exit__E
0c01b320   xdc_runtime_Core_deleteObject__I
0c01b480   xdc_runtime_Text_visitRope2__I
0c01b5e0   HeapMemMP_create
0c01b720   _buff_read
0c01bae0   fputc
0c01bae0   putc
0c01bd60   ti_sysbios_family_c64p_Hwi_Module_startup__E
0c01bd60   ti_sysbios_family_c64p_Hwi_Module_startup__F
0c01bea0   ti_sysbios_family_c66_Cache_Module_startup__E
0c01bea0   ti_sysbios_family_c66_Cache_Module_startup__F
0c01bfe0   TestApp_ReadInputData
0c01c100   __c6xabi_divlli
0c01c580   _wrt_ok
0c01c6a0   fclose
0c01c7c0   ti_sdo_ipc_heaps_HeapMemMP_Instance_finalize__F
0c01c8e0   ti_sdo_ipc_heaps_HeapMemMP_getStats__E
0c01c8e0   ti_sdo_ipc_heaps_HeapMemMP_getStats__F
0c01ca00   ti_sysbios_knl_Clock_workFunc__E
0c01cb20   ti_sysbios_knl_Task_schedule__I
0c01cc40   xdc_runtime_SysMin_flush__E
0c01cc40   xdc_runtime_SysMin_flush__F
0c01cc40   xdc_runtime_System_SupportProxy_flush__E
0c01cc40   xdc_runtime_System_flush__E
0c01cc40   xdc_runtime_System_flush__F
0c01cd60   HOSTlseek
0c01ce60   ALG_create
0c01cf60   fflush
0c01d060   ti_sdo_ipc_gates_GateHWSem_Module_startup__E
0c01d060   ti_sdo_ipc_gates_GateHWSem_Module_startup__F
0c01d160   ti_sdo_ipc_gates_GateHWSem_enter__E
0c01d160   ti_sdo_ipc_gates_GateHWSem_enter__F
0c01d260   ti_sdo_ipc_gates_GatePeterson_Object__create__S
0c01d360   ti_sdo_ipc_heaps_HeapMemMP_Object__create__S
0c01d460   ti_sdo_utils_NameServer_Module_startup__E
0c01d460   ti_sdo_utils_NameServer_Module_startup__F
0c01d560   ti_sysbios_gates_GateAll_leave__E
0c01d660   ti_sysbios_heaps_HeapMem_Object__create__S
0c01d760   ti_sysbios_knl_Semaphore_post__E
0c01d860   ti_sysbios_knl_Swi_restoreHwi__E
0c01d960   ti_sysbios_knl_Task_Object__create__S
0c01da60   ti_sysbios_knl_Task_startup__E
0c01db60   xdc_runtime_Memory_alloc__F
0c01dc60   xdc_runtime_Text_putMod__F
0c01dd60   xdc_runtime_knl_GateThread_Object__create__S
0c01de60   GateMP_close
0c01df40   HOSTopen
0c01e020   __c6xabi_divi
0c01e020   __divi
0c01e1e0   atoi
0c01e2c0   close
0c01e3a0   __TI_zero_init
0c01e480   exit
0c01e640   ltoa
0c01e720   memalign
0c01e800   memset
0c01e8e0   ti_sdo_ipc_GateMP_Object__create__S
0c01e9c0   ti_sdo_ipc_GateMP_createLocal__F
0c01eaa0   ti_sdo_ipc_gates_GateHWSem_Object__create__S
0c01eb80   ti_sysbios_gates_GateMutex_enter__E
0c01ec60   ti_sysbios_gates_GateSwi_leave__E
0c01ed40   ti_sysbios_knl_Semaphore_Object__create__S
0c01ee20   ti_sysbios_timers_timer64_Timer_stop__E
0c01efc0   GateMP_Params_init
0c01f080   HOSTread
0c01f140   HOSTunlink
0c01f200   HOSTwrite
0c01f2c0   HeapMemMP_Params_init
0c01f380   TestApp_WriteOutputData
0c01f440   _ALG_freeMemory
0c01f500   __cxa_finalize
0c01f5c0   __c6xabi_divu
0c01f5c0   __divu
0c01f680   _cleanup
0c01f740   _doflush
0c01f800   _rd_ok
0c01f8c0   ALG_delete
0c01f980   fseek
0c01fa40   lseek
0c01fb00   read
0c01fbc0   ti_sdo_ipc_MessageQ_Module_startup__E
0c01fbc0   ti_sdo_ipc_MessageQ_Module_startup__F
0c01fc80   ti_sysbios_family_c66_Cache_setMar__E
0c01fd40   ti_sysbios_heaps_HeapMem_getStats__E
0c01fe00   ti_sysbios_knl_Swi_run__I
0c01fec0   write
0c020020   HOSTclose
0c0200c0   SharedRegion_getCacheLineSize
0c020160   SharedRegion_getHeap
0c020200   SharedRegion_getId
0c0202a0   SharedRegion_isCacheEnabled
0c020340   TestApp_CompareOutputData
0c0203e0   __c6xabi_remu
0c0203e0   __remu
0c020480   _c_int00
0c0207a0   ftell
0c020840   memcpy
0c020980   ti_sdo_ipc_GateMP_getRegion0ReservedSize__F
0c020a20   ti_sdo_ipc_Notify_Object__create__S
0c020ac0   ti_sdo_ipc_gates_GatePeterson_leave__E
0c020ac0   ti_sdo_ipc_gates_GatePeterson_leave__F
0c020b60   ti_sysbios_BIOS_exitFunc__I
0c020c00   ti_sysbios_gates_GateMutexPri_Object__create__S
0c020ca0   ti_sysbios_gates_GateMutex_Object__create__S
0c020d40   ti_sysbios_gates_GateSwi_enter__E
0c020de0   ti_sysbios_knl_Clock_Instance_finalize__F
0c020e80   ti_sysbios_knl_Task_Params__init__S
0c020f20   ti_sysbios_xdcruntime_GateThreadSupport_Object__create__S
0c020fc0   xdc_runtime_Error_print__E
0c020fc0   xdc_runtime_Error_print__F
0c021060   xdc_runtime_System_abort__E
0c021060   xdc_runtime_System_abort__F
0c021100   xdc_runtime_Text_xprintf__I
0c0211a0   GateMP_enter
0c021220   GateMP_leave
0c021320   TestApp_EnableCache
0c0213a0   _Z11__TI_atexitPFYvPvES_S_
0c0213a0   __cxa_atexit
0c021420   __c6xabi_llshl
0c0214a0   ti_sysbios_family_c62_TaskSupport_swap__E
0c021520   fprintf
0c0215a0   malloc
0c021620   printf
0c0216a0   readmsg
0c021720   strncpy
0c0217a0   ti_sdo_ipc_Notify_Module_startup__E
0c0217a0   ti_sdo_ipc_Notify_Module_startup__F
0c021820   ti_sysbios_family_c66_Cache_wbInvAll__E
0c0218a0   ti_sysbios_gates_GateAll_Object__create__S
0c021920   ti_sysbios_hal_Hwi_checkStack
0c0219a0   ti_sysbios_knl_Idle_loop__E
0c021a20   ti_sysbios_knl_Semaphore_pendTimeout__I
0c021aa0   ti_sysbios_knl_Swi_post__E
0c021b20   ti_sysbios_knl_Task_unblockI__E
0c021ba0   remove
0c021ba0   unlink
0c021c20   xdc_runtime_Assert_raise__I
0c021ca0   xdc_runtime_Startup_exec__E
0c021ca0   xdc_runtime_Startup_exec__F
0c021d20   xdc_runtime_System_rtsExit__I
0c021da0   xdc_runtime_Text_printVisFxn__I
0c021e20   xdc_runtime_knl_GateThread_Instance_finalize__F
0c021ea0   __c6xabi_frcmpyd_div
0c021f00   __c6xabi_llshru
0c021f60   __c6xabi_remull
0c021fc0   _subcull
0c022020   fopen
0c022080   memccpy
0c0220e0   memcmp
0c0221a0   sscanf
0c022200   ti_sdo_ipc_gates_GateHWSem_Object__delete__S
0c022260   ti_sdo_ipc_gates_GateMPSupportNull_Object__create__S
0c0222c0   ti_sdo_ipc_gates_GateMPSupportNull_Object__delete__S
0c022320   ti_sdo_ipc_gates_GatePeterson_Instance_finalize__F
0c022380   ti_sdo_ipc_gates_GatePeterson_Object__delete__S
0c0223e0   ti_sdo_ipc_gates_GatePeterson_sharedMemReq__E
0c0223e0   ti_sdo_ipc_gates_GatePeterson_sharedMemReq__F
0c022440   ti_sdo_ipc_heaps_HeapMemMP_Object__delete__S
0c0224a0   ti_sdo_utils_List_Object__create__S
0c022500   ti_sysbios_family_c64p_Exception_Module_startup__E
0c022500   ti_sysbios_family_c64p_Exception_Module_startup__F
0c022560   ti_sysbios_family_c66_Cache_setSize__E
0c0225c0   ti_sysbios_gates_GateAll_Object__delete__S
0c022620   ti_sysbios_gates_GateAll_enter__E
0c022680   ti_sysbios_gates_GateMutexPri_Object__delete__S
0c0226e0   ti_sysbios_gates_GateMutex_Object__delete__S
0c022740   ti_sysbios_gates_GateSwi_Object__create__S
0c0227a0   ti_sysbios_gates_GateSwi_Object__delete__S
0c022800   ti_sysbios_hal_Hwi_initStack
0c022860   ti_sysbios_heaps_HeapMem_Object__delete__S
0c0228c0   ti_sysbios_knl_Clock_doTick__I
0c022920   ti_sysbios_knl_Queue_Object__create__S
0c022980   ti_sysbios_knl_Task_Module_startup__E
0c022980   ti_sysbios_knl_Task_Module_startup__F
0c0229e0   ti_sysbios_knl_Task_allBlockedFunction__I
0c022a40   ti_sysbios_knl_Task_enter__I
0c022aa0   writemsg
0c022af8   C$$IO$$
0c022b00   xdc_runtime_GateNull_Object__create__S
0c022b60   xdc_runtime_GateNull_Object__delete__S
0c022bc0   xdc_runtime_Memory_calloc__E
0c022bc0   xdc_runtime_Memory_calloc__F
0c022c20   xdc_runtime_SysMin_putch__E
0c022c20   xdc_runtime_SysMin_putch__F
0c022c80   xdc_runtime_System_atexit__E
0c022c80   xdc_runtime_System_atexit__F
0c022ce0   xdc_runtime_knl_GateThread_Object__delete__S
0c022d40   __c6xabi_isinf
0c022dc0   _args_main
0c022e00   ti_sysbios_family_c62_TaskSupport_buildTaskStack
0c022e40   ti_sysbios_family_xxx_Hwi_switchToIsrStack
0c022e80   free
0c022ec0   llabs
0c022f00   main
0c022f40   readparamfile
0c022fc0   strcmp
0c023000   strlen
0c023040   ti_sdo_ipc_gates_GateHWSem_Handle__label__S
0c023080   ti_sdo_ipc_gates_GateHWSem_leave__E
0c023080   ti_sdo_ipc_gates_GateHWSem_leave__F
0c0230c0   ti_sdo_ipc_gates_GateMPSupportNull_Handle__label__S
0c023100   ti_sdo_ipc_gates_GateMPSupportNull_enter__E
0c023100   ti_sdo_ipc_gates_GateMPSupportNull_enter__F
0c023140   ti_sdo_ipc_gates_GatePeterson_Handle__label__S
0c023180   ti_sdo_ipc_heaps_HeapMemMP_Handle__label__S
0c0231c0   ti_sysbios_gates_GateAll_Handle__label__S
0c023200   ti_sysbios_gates_GateMutexPri_Handle__label__S
0c023240   ti_sysbios_gates_GateMutexPri_Instance_finalize__F
0c023280   ti_sysbios_gates_GateMutex_Handle__label__S
0c0232c0   ti_sysbios_gates_GateMutex_Instance_finalize__F
0c023300   ti_sysbios_gates_GateSwi_Handle__label__S
0c023340   ti_sysbios_hal_Hwi_Module_startup__E
0c023340   ti_sysbios_hal_Hwi_Module_startup__F
0c023380   ti_sysbios_hal_Timer_Module_startup__E
0c023380   ti_sysbios_hal_Timer_Module_startup__F
0c0233c0   ti_sysbios_heaps_HeapMem_Handle__label__S
0c023400   ti_sysbios_heaps_HeapMem_init__I
0c023440   ti_sysbios_knl_Clock_Module_startup__E
0c023440   ti_sysbios_knl_Clock_Module_startup__F
0c023480   ti_sysbios_knl_Semaphore_Instance_finalize__F
0c023540   ti_sysbios_xdcruntime_GateThreadSupport_Instance_finalize__F
0c023580   TSC_enable
0c023588   TSC_read
0c0235c0   xdc_runtime_GateNull_Handle__label__S
0c023600   xdc_runtime_Memory_free__E
0c023600   xdc_runtime_Memory_free__F
0c023640   xdc_runtime_SysMin_Module_startup__E
0c023640   xdc_runtime_SysMin_Module_startup__F
0c023680   xdc_runtime_System_aprintf__E
0c0236c0   xdc_runtime_System_printf__E
0c023700   xdc_runtime_knl_GateThread_Handle__label__S
0c0237a0   TestApp_SetDynamicParams
0c0237c0   TestApp_SetInitParams
0c0237e0   __c6xabi_negll
0c023800   __cxa_ia64_exit
0c023820   __xdc__init
0c023860   _nop
0c023900   _register_lock
0c023920   _register_unlock
0c023940   ti_sysbios_family_c62_TaskSupport_glue
0c023960   ti_sysbios_family_xxx_Hwi_switchToTaskStack
0c0239a0   C$$EXIT
0c0239a0   abort
0c0239c0   atexit
0c0239e0   __TI_decompress_none
0c023a00   __TI_decompress_rle24
0c023a20   feof
0c023a40   fgets
0c023a60   ti_sdo_ipc_gates_GateHWSem_getReservedMask__E
0c023a60   ti_sdo_ipc_gates_GateHWSem_getReservedMask__F
0c023a80   ti_sdo_ipc_gates_GateHWSem_query__E
0c023a80   ti_sdo_ipc_gates_GateHWSem_query__F
0c023aa0   ti_sdo_ipc_gates_GateHWSem_sharedMemReq__E
0c023aa0   ti_sdo_ipc_gates_GateHWSem_sharedMemReq__F
0c023ac0   ti_sdo_ipc_gates_GateMPSupportNull_getReservedMask__E
0c023ac0   ti_sdo_ipc_gates_GateMPSupportNull_getReservedMask__F
0c023ae0   ti_sdo_ipc_gates_GateMPSupportNull_leave__E
0c023ae0   ti_sdo_ipc_gates_GateMPSupportNull_leave__F
0c023b00   ti_sdo_ipc_gates_GateMPSupportNull_query__E
0c023b00   ti_sdo_ipc_gates_GateMPSupportNull_query__F
0c023b20   ti_sdo_ipc_gates_GateMPSupportNull_sharedMemReq__E
0c023b20   ti_sdo_ipc_gates_GateMPSupportNull_sharedMemReq__F
0c023b40   ti_sdo_ipc_gates_GatePeterson_getReservedMask__E
0c023b40   ti_sdo_ipc_gates_GatePeterson_getReservedMask__F
0c023b60   ti_sdo_ipc_gates_GatePeterson_query__E
0c023b60   ti_sdo_ipc_gates_GatePeterson_query__F
0c023b80   ti_sdo_ipc_heaps_HeapMemMP_isBlocking__E
0c023b80   ti_sdo_ipc_heaps_HeapMemMP_isBlocking__F
0c023ba0   ti_sysbios_BIOS_start__E
0c023bc0   ti_sysbios_family_c66_Cache_getMar__E
0c023be0   ti_sysbios_family_c66_Cache_wbInv__E
0c023c00   ti_sysbios_gates_GateAll_query__E
0c023c00   ti_sysbios_gates_GateAll_query__F
0c023c20   ti_sysbios_gates_GateMutexPri_query__E
0c023c20   ti_sysbios_gates_GateMutexPri_query__F
0c023c20   ti_sysbios_xdcruntime_GateThreadSupport_query__E
0c023c20   ti_sysbios_xdcruntime_GateThreadSupport_query__F
0c023c20   xdc_runtime_knl_GateThread_Proxy_query__E
0c023c20   xdc_runtime_knl_GateThread_query__E
0c023c20   xdc_runtime_knl_GateThread_query__F
0c023c40   ti_sysbios_gates_GateMutex_leave__E
0c023c60   ti_sysbios_gates_GateMutex_query__E
0c023c60   ti_sysbios_gates_GateMutex_query__F
0c023c80   ti_sysbios_gates_GateSwi_query__E
0c023c80   ti_sysbios_gates_GateSwi_query__F
0c023ca0   ti_sysbios_heaps_HeapMem_isBlocking__E
0c023cc0   ti_sysbios_knl_Swi_Module_startup__E
0c023cc0   ti_sysbios_knl_Swi_Module_startup__F
0c023ce0   xdc_runtime_GateNull_enter__E
0c023ce0   xdc_runtime_GateNull_enter__F
0c023d00   xdc_runtime_GateNull_leave__E
0c023d00   xdc_runtime_GateNull_leave__F
0c023d20   xdc_runtime_GateNull_query__E
0c023d20   xdc_runtime_GateNull_query__F
0c023d60   xdc_runtime_Startup_exec__I
0c023d80   xdc_runtime_Startup_reset__I
0c023da0   xdc_runtime_System_Module_startup__E
0c023da0   xdc_runtime_System_Module_startup__F
0c023dc0   xdc_runtime_System_exit__E
0c023dc0   xdc_runtime_System_exit__F
0c023de0   xdc_runtime_Text_visitRope__I
0c023e00   xdc_runtime_knl_GateThread_enter__E
0c023e00   xdc_runtime_knl_GateThread_enter__F
0c023e20   xdc_runtime_knl_GateThread_leave__E
0c023e20   xdc_runtime_knl_GateThread_leave__F
0c024000   ti_sysbios_family_c64p_Hwi0
0c024020   ti_sysbios_family_c64p_Hwi1
0c024040   ti_sysbios_family_c64p_Hwi2
0c024060   ti_sysbios_family_c64p_Hwi3
0c024080   ti_sysbios_family_c64p_Hwi4
0c0240a0   ti_sysbios_family_c64p_Hwi5
0c0240c0   ti_sysbios_family_c64p_Hwi6
0c0240e0   ti_sysbios_family_c64p_Hwi7
0c024100   ti_sysbios_family_c64p_Hwi8
0c024120   ti_sysbios_family_c64p_Hwi9
0c024140   ti_sysbios_family_c64p_Hwi10
0c024160   ti_sysbios_family_c64p_Hwi11
0c024180   ti_sysbios_family_c64p_Hwi12
0c0241a0   ti_sysbios_family_c64p_Hwi13
0c0241c0   ti_sysbios_family_c64p_Hwi14
0c0241e0   ti_sysbios_family_c64p_Hwi15
80000000   ti_sdo_utils_NameServer_Module_State_0_nsRemoteHandle__A
80000008   ti_sysbios_heaps_HeapMem_Instance_State_0_buf__A
81f0f010   ti_sysbios_knl_Task_Instance_State_0_hookEnv__A
81f0f020   xdc_runtime_SysMin_Module_State_0_outbuf__A
81f14240   internalDataMemory
81f16240   params
81f16258   dynamicParams
81f16278   inArgs
81f1627c   outArgs
81f1628c   status
81f1632c   InBuffers
81f163f0   OutBuffers
81f164c0   InputBuffSize
81f164d0   _tmpnams
81f166f0   inputData
8229a6f0   outputData
822ba700   refData
ffffffff   __TI_pprof_out_hndl
ffffffff   __TI_prof_data_size
ffffffff   __TI_prof_data_start
ffffffff   __binit__
ffffffff   binit

[613 symbols]
